:106D6C000000050200000301FA0400EF0500030A0D
:106D7C000A5A0B001E0C00FA0D00030E00040F0142
:106D8C0064100096120132130AFA14010217010A58
:106D9C001801EF1905321A010A1B01EF1C05321FED
:106DAC00FFFF20FFFF23011E2400642A00FA2B00A2
:106DBC00FA2C50782D003D2E00463000643250786D
:106DCC003300003432FA350164360164370150382F
:106DDC000A643A00033B00043C00643E003C3F0064
:106DEC000140FFFF411450420A5A430AC84405327D
:106DFC004500B44600FA4900024B00014C00FA5021
:106E0C000606510596520A32530B46540A965705FC
:106E1C0046590A465A32FA5B010A5C0A325E000A8B
:106E2C005F00646200FE64021C67FFFF6801016979
:106E3C0001016A05966B00006C32966D00047300BC
:106E4C00007400007801327901327E0064810064A4
:106E5C0084FFFF8800028A00019D0A969E00019F14
:106E6C00FFFFA0013CA2000AA3FFFFA4FFFFA5FFA8
:106E7C00FFA6FFFFA7FFFFA8FFFFA9FFFF01013C33
:106E8C001500022F003C4701784802045602024EBE
:106E9C00FFFF58000261FFFF6600028500AF86000D
:106EAC00018700FA890108990006A100FAFAFAFA9A
:106EBC0001013C1500022F1E3C4701784802045684
:106ECC0002024EFFFF58000261FFFF6600028500C0
:106EDC00AF8600018700FA890108990000A1000023
:106EEC00FAFAFA0065006F00790083008D009700B4
:106EFC00A100AC00B600C000CA00D400DE00E8005F
:106F0C00F200580060006800700078008000880073
:106F1C0090009800A000A800B000B800C100C80004
:106F2C00D000D800DF00E600EE00F600410047007C
:106F3C004D00530059005F0065006C007100770034
:106F4C007D00830089008F0095009B00A200A700A4
:106F5C00AC00B200B900C000C500CA00D200D50018
:076F6C00DD00E100E700EF8A
:103CD80075A71085F97385FA747E017F00E5741263
:103CE8007085E5732FFF50010E8E598F5A9000187A
:103CF800E0FCA3E0FDEF2DFDEE3CFC8C5B8D5C90C1
:103D08000038E0FAA3E0FBED2BFBEC3AFA8A5B8B78
:103D18005C2275A71085F97385FA747E017F00E52A
:103D280074127085E5732FFF50010E8E598F5AACAF
:103D38002CAD2DEF2DFDEE3CFC8C5B8D5C9000389E
:103D4800E0FAA3E0FBED2BFBEC3AFA8A5B8B5C22F2
:103D5800E55CF5FBE55BF5FCD29322E55CF5E9E56E
:103D68005BF5EAD29422E55CF5EBE55BF5ECD291E4
:103D780022E55CF5EDE55BF5EED29222E55CF5FD1A
:103D8800E55BF5FED28722E55CF5CEE55BF5CFD2A3
:103D98009022A203B34004D2978002C29722E50C76
:103DA80090695BF8282873806CA237B34008E5B5A2
:103DB8004408F5B58006E5B554F7F5B58057A23740
:103DC800B34008E5B54402F5B58006E5B554FDF500
:103DD800B58042A2379297803CA237B34008E5B538
:103DE8004410F5B58006E5B554EFF5B58027A23740
:103DF800B34008E5B54420F5B58006E5B554DFF5D0
:103E0800B58012A2379292800CA23792878006A2C0
:053E18003792908000CC
:10695B00023DAF023DB1023DC6023DDB023DE1020D
:0E696B003DF6023E0B023E11023E17023E1D9B
:103E1D0022743690015FF07430900160F0742D9033
:103E2D000161F07432900162F07420900163F074BE
:103E3D0042900164F0744D900165F07457900166E5
:103E4D00F07420900167F0744D900168F074339018
:103E5D000169F0742090016AF0744590016BF07463
:103E6D003490016CF0743690016DF022900896E05C
:103E7D00FEA3E0FF741DD39F74019E400C906D6CEA
:103E8D00120048E493F599802E90F802E493B4055E
:103E9D0014900896E0FEA3E0FF906D9F120048E499
:103EAD0093F5998012900896E0FEA3E0FF906D6C5B
:103EBD00120048E493F59990089612709390089625
:103ECD00E0FEA3E0FFEFB45007EEB40103754D0023
:103EDD0022AE59AF5A74068E048F05FF1270758C81
:103EED005B8D5CAE59AF5A74068E048F05FF127050
:103EFD00A08C598D5AE55A455960137406C3955ACD
:103F0D00FFE49559FE8E598F5A785B1270D8E57380
:103F1D00A85BB80015D3955C4010E573C3955CFFA5
:103F2D00E4955BFE8E5B8F5C8010E573243CC3953E
:103F3D005CFFE4955BFE8E5B8F5CAE5BAF5C743BB0
:103F4D006F4E6006743C6F4E701AAE5BAF5C743B87
:103F5D006F4E70057573018003757302755C3A754C
:103F6D005B0080037573002290009CE0B40104C2D5
:103F7D00078002D20790009DE0B40104C2088002C0
:103F8D00D2089000DAE075F0D2A4FFAEF0740A8E7C
:103F9D00048F05FF12707590088AECF0A3EDF09078
:103FAD0000DAE075F02BA4FFAEF0900014EEF0A354
:103FBD00EFF07E017F00900098E01270859000DB9D
:103FCD00E08E048F05FF127075740AFF1270758DE7
:103FDD00609000E4E075F0D2A4FFAEF0740A8E0498
:103FED008F05FF12707590088EECF0A3EDF0900028
:103FFD00E6E060139000E6E0F5F0741684FF7E00B5
:10400D00EF9008ECF0800674649008ECF09000DC02
:10401D00E0900077F0900128E0900083F090012A65
:10402D00E0FE9000D8E08E0088F0A4FFAEF0EF9097
:10403D0008F5F0900103E075F013A4FDACF09000CD
:10404D0038ECF0A3EDF0A220B34016900174E070AF
:10405D000C900175E07006900176E060028002C25E
:10406D0020900174E0B4300F900175E0B4470890D2
:10407D000176E0643B60028004D2218002C221748B
:10408D00E3900076F09000C5E0B40B0874E3900067
:10409D0076F0805A9000C5E0B419129000DBE090E4
:1040AD006EDA12008CE493900076F080419000C59A
:1040BD00E0B41E129000DBE0906EF812008CE493D9
:1040CD00900076F080289000C5E0B428129000DBB7
:1040DD00E0906F2212008CE493900076F0800F90A8
:1040ED0000C5E0B446089000BCE0900076F090006A
:1040FD0095E0FE9008F6E06E601A7599E612019C47
:10410D0074AB900050F012069A7509647508001290
:10411D0005E480FE90008DE0700674009000C2F002
:10412D0090007BE0FE9000C2E0B5065790007DE068
:10413D00FE9000E0E0B5064B90007CE0FE9000EEB6
:10414D00E0B5063F900081E0FE900095E0B50633A6
:10415D0090007EE0FE9000D0E0B5062790007FE055
:10416D00FE9000FBE0B5061B900080E0FE9000FC89
:10417D00E0B5060F900082E0FE90010EE06E700338
:10418D0002436A90009DE070089000DEE0640460D8
:10419D0002800674039000DEF09000D0E0D394020C
:1041AD0050069000EEE060087405900111F0800655
:1041BD007408900111F0900095E0B4010674009020
:1041CD000095F0900095E0B4020674009000E0F0C8
:1041DD00900095E0B4030674009000EDF090010E90
:1041ED00E06014742A900786F074009006D2F07483
:1041FD00009006D3F0800C7400900786F0742A901E
:10420D0006D2F09000E0E0D39401401A74189001AA
:10421D0013F07400900114F074009006D6F0740041
:10422D009006D7F0803D9000EEE0B401089000D0EC
:10423D00E064036002801A7400900113F07418900A
:10424D000114F074009006D6F074009006D7F0803B
:10425D00127400900113F07400900114F074189012
:10426D0006D6F09000C2E0601474079000A9F074B7
:10427D00009006DAF074009006DBF0800C7400906C
:10428D0000A9F074079006DAF09000C2E0B40214B1
:10429D0074089000AAF074009006DEF07400900689
:1042AD00DFF0800C74009000AAF074089006DEF028
:1042BD009000D0E0B402069000EEE060028026741B
:1042CD00049006E2F074059006E6F074069006EA96
:1042DD00F07400900781F07400900782F0740090E4
:1042ED000783F0803674009006E2F074009006E3C8
:1042FD00F074009006E6F074009006E7F0740090FC
:10430D0006EAF074009006EBF07404900781F074E7
:10431D0005900782F07406900783F0D21F9000C2BB
:10432D00E090007BF09000EEE090007CF09000E0DB
:10433D00E090007DF09000D0E090007EF090009530
:10434D00E0900081F09000FBE090007FF09000FC89
:10435D00E0900080F090010EE0900082F09000F867
:10436D00E0B40117900024740FF0A374FFF09000D7
:10437D0026E4F0A3F074029000F8F09000F8E0B499
:10438D000341900026E0FEA3E0FF900024E0FCA393
:10439D00E0FD1270D074101270857408120039EFA0
:1043AD009000F7F0EF700674FF9000F7F074009036
:1043BD0000F8F0900025E09000AEF0900024E09021
:1043CD0000AFF0900089E0900086F0900088E090BA
:1043DD000085F09000B7E0C3941E50569000B7E0F2
:1043ED00F404241E900087F0900087E075F0068499
:1043FD00FF7E008F73900087E075F00684ADF07C32
:10440D00008D74900085E0D39574400D900085E08B
:10441D00C39574900085F0800F900085E02406C34D
:10442D009574900085F00573900086E025739000DB
:10443D0086F0900086E0900046F0900046E024144F
:10444D00900047F0900046E02428900048F090003E
:10445D0047E0D3943C400B900047E0C3943C900060
:10446D0047F0900048E0D3943C400B900048E0C3E7
:10447D00943C900048F090004CE4F0900046E064CD
:10448D003B6007900046E0B43C20900046E0B43B12
:10449D0006740290004CF0900046E0B43C0690008B
:1044AD004C7401F09000467401F090004DE4F090D2
:1044BD000047E0643B6007900047E0B43C2090006B
:1044CD0047E0B43B06740290004DF0900047E0B415
:1044DD003C0690004D7401F09000477401F090007F
:1044ED004EE4F0900048E0643B6007900048E0B473
:1044FD003C20900048E0B43B06740290004EF090D2
:10450D000048E0B43C0690004E7401F090004874F1
:10451D0001F0900089E0FE9000ECE02E900051F04B
:10452D00900051E0D3943C400B900051E0C3943C7B
:10453D00900051F0900051E0D3943C400B9000510D
:10454D00E0C3943C900051F09000C7E0B40163903B
:10455D000051E0641E6007900051E0B43C069000ED
:10456D0051E004F0900051E0641D6007900051E0AF
:10457D00B43B06900051E014F0900051E0D3943C10
:10458D00400B900051E0C3943C900051F0900051CD
:10459D00E0D3941E400D900051E0C3941E90005244
:1045AD00F0800A900051E0241E900052F0755D1EBF
:1045BD008079900051E06414600F900051E0642800
:1045CD006007900051E0B43C06900051E004F0907B
:1045DD000051E06413600F900051E0642760079074
:1045ED000051E0B43B06900051E014F0900051E012
:1045FD00D3943C400B900051E0C3943C900051F09B
:10460D00900051E0D39414400B900051E0C39414EA
:10461D00900051F0900051E0D39414400B90005154
:10462D00E0C39414900051F0755D14900089E0FE84
:10463D009000CFE0D39E5013900089E0FE9000CF04
:10464D00E0F4042E04900049F08013900089E024DA
:10465D0078FE9000CFE0F4042E04900049F0900015
:10466D0049E075F01484AFF07E00EF4E70069000B7
:10467D0049E004F0900049E00475F01484AFF07E39
:10468D0000EF4E7006900049E014F0900049E0B440
:10469D0079069000497401F0900049E0D3943C40B4
:1046AD000F900049E0C3943C900049F0D21A80026B
:1046BD00C21A900049E0241490004AF0900049E09D
:1046CD00242890004BF090004AE0D3943C400B908E
:1046DD00004AE0C3943C90004AF090004BE0D39424
:1046ED003C400B90004BE0C3943C90004BF012010A
:1046FD009C22C293C294C291C292C287C290E5B568
:10470D0054EFF5B5E5B554DFF5B5C296C295C2A027
:10471D00C297C2A2C2A1E5B554BFF5B5E5B5547FA8
:10472D00F5B5E5B554FBF5B5C209755E469000D2F9
:10473D00E07005756D028003756D0375540075533A
:10474D000090000C74FFF0A374DCF0C20FC211C214
:10475D001374C890003AF074C890003EF074C8907D
:10476D000042F0755200755100C204754600E56FA8
:10477D00B41303756F0075630090001AE4F0A3F095
:10478D00757010C20CC20DC20EC203755600755560
:10479D000090000EE4F0A3F0900010E4F0A3F0C23E
:1047AD0027755800755700900094E075F032A4FFFE
:1047BD00AEF0900022EEF0A3EFF0900084E4F090C4
:1047CD0008F2E4F0C222C218C219C21AC21B90002C
:1047DD0012E4F0A3F022755A00755900AE59AF5A84
:1047ED00741CC39F74019E50030248D7906D6C12C8
:1047FD000048E493645F6023906D6C120048E4936D
:10480D00647E6017906D6C120048E4936481600BB8
:10481D00906D6C120048E493B484030248B7AE590E
:10482D00AF5A906D6C120048E4939000881270B6E8
:10483D000FBF00010EE0FC906D6C120048ECFEE421
:10484D0093FFEEC39F5026AE59AF5A0FBF00010E16
:10485D00906D6C120048AE59AF5AE493FC906D6C9C
:10486D00120048E4939000881270B6ECF0AE59AF88
:10487D005A906D6C120048E4939000881270B6E067
:10488D00FC906D6E120048ECFCE493FDECD39D4062
:10489D0019906D6E120048E493FC906D6C120048F7
:1048AD00E4939000881270B6ECF0AE59AF5A7402D2
:1048BD002FFF50010E8E598F5A785A740126F650DB
:1048CD000418E436F640030247E922755A0075597B
:1048DD0000AE59AF5A7432BE00039F50030249A572
:1048ED00906E89120048E4939000881270B60FBF45
:1048FD0000010EE0FC906E89120048ECFEE493FF7F
:10490D00EEC39F5026AE59AF5A0FBF00010E906EE9
:10491D0089120048AE59AF5AE493FC906E8912008B
:10492D0048E4939000881270B6ECF0AE59AF5A90EF
:10493D006E89120048E4939000881270B6E0FC90E6
:10494D006E8B120048ECFCE493FDECD39D40199066
:10495D006E8B120048E493FC906E89120048E4932C
:10496D009000881270B6ECF0AE59AF5A742D6F4EA0
:10497D007006755A33755900AE59AF5A74022FFF30
:10498D0050010E8E598F5A785A740126F65004181C
:10499D00E436F640030248DE22755A00755900AE22
:1049AD0059AF5A7432BE00039F5003024A73906E82
:1049BD00BC120048E4939000881270B60FBF00013E
:1049CD000EE0FC906EBC120048ECFEE493FFEEC3CB
:1049DD009F5026AE59AF5A0FBF00010E906EBC12FC
:1049ED000048AE59AF5AE493FC906EBC120048E4F7
:1049FD00939000881270B6ECF0AE59AF5A906EBC21
:104A0D00120048E4939000881270B6E0FC906EBEE0
:104A1D00120048ECFCE493FDECD39D4019906EBE62
:104A2D00120048E493FC906EBC120048E493900091
:104A3D00881270B6ECF0AE59AF5A742D6F4E7006E9
:104A4D00755A33755900AE59AF5A74022FFF500184
:104A5D000E8E598F5A785A740126F6500418E43682
:104A6D00F640030249AC2275A71085F97385FA74D7
:104A7D007E017F00E574127085E5732FFF50010EE6
:104A8D008E598F5AAC5BAD5CEF2DFDEE3CFC8C5B13
:104A9D008D5C123D58123D63123D6E9000D0E0D3F7
:104AAD0094024009123D79123D84123D8F75A70085
:104ABD002285F97385FA747E017F00E57412708585
:104ACD00E5732FFF50010E8E598F5A7E017F769020
:104ADD00010DE0127085AC59AD5AED2FFFEC3EFE85
:104AED008E5B8F5CE55CF5EDE55BF5EE900077E4B4
:104AFD00F07412900054F02285F97385FA747E01DA
:104B0D007F00E574127085E5732FFF50010E8E59ED
:104B1D008F5A900014E0FCA3E0FDEF2DFDEE3CFC60
:104B2D008C5B8D5CE55CF5FDE55BF5FE2205642295
:104B3D00A2DBB340089000DCE0900077F0A2DCB37C
:104B4D004024A29650067419900054F0A295500678
:104B5D007419900054F0A2A050067419900054F0EE
:104B6D00C296C295C2A075D8402285A77275A710AE
:104B7D009000D0E0D3940250079000EEE0B40252C2
:104B8D00A2D8B34002C293A2D9B34002C294A2DA12
:104B9D00B34002C2919000D0E0640260079000D053
:104BAD00E0B40417A2DBB34002C292A2DCB3400210
:104BBD00C287A2DDB34002C2908015A2D8B34002D5
:104BCD00C292A2D9B34002C287A2DAB34002C29008
:104BDD00802DA2D8B3400AC2939000EEE06002C2CD
:104BED0092A2D9B3400AC2949000EEE06002C2874F
:104BFD00A2DAB3400AC2919000EEE06002C2907555
:104C0D00D8408572A72290F800E493640660028074
:104C1D00FE12009E75A70075D80075D90475DD09C3
:104C2D0075DE0975D84075A71075D80075D904754E
:104C3D00DA0975DB0975DC0975DD0975DE0975DFC6
:104C4D000975D84075A7001200FB7509C8750800D5
:104C5D001205E475A70FE5FC900063F0E5FB9000ED
:104C6D0064F0E5FA900065F0E5F9900066F075A73F
:104C7D000090F800E493F52712070390089FE0D306
:104C8D009403500790089FE0B40106740090089FAC
:104C9D00F090089FE09008F6F074019000D1F0902C
:104CAD00089FE0906979F8282873802A802875A7D5
:104CBD000F75F30F75A700A2A3400674029000D1E3
:104CCD00F0801375A70F75F31775A700A2A4400602
:064CDD0074029000D1F00A
:0C697900024CB7024CB9024CBB024CD0DF
:104CE3009000D1E0B4022AC217120AAC74029000F9
:104CF300D1F090089FE0906985F828287380108090
:0F4D03000E74009000E0F0800674009000EDF058
:0C698500024D00024D02024D04024D0CB8
:104D12008028D2171209C174019000D1F090089F27
:104D2200E0906991F82828738010800E740090003A
:0A4D3200E0F0800674009000EDF040
:0C699100024D2A024D2C024D2E024D3604
:104D3C0090F807E493900070F0900070E0440890B5
:104D4C000070F0900070E054FE900070F012039D23
:104D5C00123E1E9008ACE0900174F09008ADE0900B
:104D6C000175F09008AEE0900176F0900174E0705F
:104D7C000C900175E07006900176E060028004C230
:104D8C00208002D2209000C2E00490007BF01247F9
:104D9C00E390F802E493B405051249A68003124887
:104DAC00D874009000F8F0123F75E5B54401F5B5E4
:104DBC007406900056F07400900057F07401900047
:104DCC0058F090F802E493900059F090F803E493B3
:104DDC0090005AF090F804E49390005BF074069005
:104DEC00005CF0900059E0B40506740590005CF08E
:104DFC00744690005DF0740390005EF074069000B1
:104E0C005FF07407900060F090F805E493900061F7
:104E1C00F090F806E493900062F0740090006AF051
:104E2C00740090006BF0740090006CF074009000B3
:104E3C006DF0740090006EF0740090006FF074FFD1
:104E4C00900071F0A2B6B39205A2B3B39206A2A4DD
:104E5C00B3921DA2A3B3921E900072E4F0756F0082
:104E6C00743A900788F074FD900789F0900073E411
:104E7C00F0756E01900054E4F09000D2E0B401069D
:104E8C00741A900054F0C21C756300C20AD20BC293
:104E9C0003757100C21F120586755F00756B007576
:104EAC006100756532756600756700756800756917
:104EBC0000756A0090001AE4F0A3F0756C00D2B291
:104ECC00D2A4D2B0D2B1D2A3D2A7D2A6D2A5D2B7F5
:104EDC007E017F009000AFE01270859000AEE02F55
:104EEC00FF50010E900024EEF0A3EFF0EFD394FFEF
:104EFC00EE940F4007900024E4F0A3F09000F7E04C
:104F0C00700674FF9000F7F09000D2E07005756D9C
:104F1C00028003756D03741C900115F0741A9001D6
:104F2C0016F07400900117F07400900118F07429B9
:104F3C009006CEF07415900776F07416900777F003
:104F4C007417900778F07400900779F0740090074C
:104F5C007AF0740090077BF0740090077CF074007A
:104F6C0090077DF0740190077EF0740290077FF03B
:104F7C007403900780F07400900784F0740090071D
:104F8C0085F0D29CE570D394104003757010900698
:104F9C00CFE0D3940C400674009006CFF09006D36B
:104FAC00E0D3940C400674009006D3F09006D7E042
:104FBC00D3940C400674009006D7F09006DBE0D337
:104FCC00940C400674009006DBF09006DFE0D3945E
:104FDC000C400674009006DFF09006E3E0D3940CCE
:104FEC00400674009006E3F09006E7E0D3940C4082
:104FFC000674009006E7F09006EBE0D3940C4006A4
:10500C0074009006EBF0D2EC75CF01A298B340057A
:10501C00C298120C14E54D6006A299B3B3400280FD
:10502C0005C2991210A3E54E64016005E54EB40467
:10503C000280D5C28E7E107F00E564127085E58DEE
:10504C0075F010A4FDACF0EF2DFDEE3CFCE58B757E
:10505C00F01084FF7E00ED2FFFEC3EFE8E538F543C
:10506C00D28E9000B5E060099000B5E0C3943D404D
:10507C0002805690001C12709390001CE0FEA3E07E
:10508C00FF90001EE0FCA3E0FDEFB5053CEEB5047F
:10509C0038B215A204B34013A215B34008E5B544C9
:1050AC0004F5B58006E5B554FBF5B590001EE0FEA1
:1050BC00A3E0FF900020E0FCA3E0FDEF2DFDEE3C13
:1050CC00FC90001EECF0A3EDF09000C2E0600990A3
:1050DC0000C2E0C3940340028077122FCEA204409A
:1050EC00089000ACE0F545801BE55FC3956050056A
:1050FC00754500800F900099E0C3956150069000B3
:10510C00BFE0F545E54575F002A4FFAEF0900894BC
:10511C00EEF0A3EFF0AC2EAD2FEDD39FEC9E40152F
:10512C00E5B554EFF5B59000C2E0B40206E5B54420
:10513C0020F5B5801C900072E0C394415013E5B586
:10514C004410F5B59000C2E0B40206E5B554DFF5A5
:10515C00B59000C2E0B403241230E9AE2EAF2F900C
:10516C000894E0FCA3E0FDEFD39DEE9C4008E5B570
:10517C0054EFF5B58006E5B54410F5B590009DE00B
:10518C006009A2B3300601B3B340028039A2B33038
:10519C000601B34031A2B3300801B3401C9000D0DB
:1051AC00E0B40306A218B3B3400280067405900065
:1051BC0054F0D218A208B39206A208B330B301B3CC
:1051CC004004A2089206A2B6300501B35003025760
:1051DC00A1A2B6300501B350030257A1A2B6300705
:1051EC0001B350030256BF756E009000B5E0B43D9C
:1051FC0013A207B34008E5B554FBF5B58006E5B539
:10520C004404F5B5055EA209B3B35013AE53AF54C5
:10521C0090000CE0FCA3E0FDEDC39FEC9E4003026C
:10522C005372E56DB4032EA227B34022E55EB43B66
:10523C0003756D01E55EC3943B50069000547401F8
:10524C00F0E55ED3943B40067402900054F0755E1A
:10525C0001D227805CE56DB40206756D01755E3B6D
:10526C00E55EB43B05755E018047900054E07032FA
:10527C00E55EC3943B50069000547401F0E55ED398
:10528C00943B40067402900054F0E55EC3943B508E
:10529C0002D21CE55ED3943B4002D21CC296C2954E
:1052AC00C2A09000D2E0B401051246FF8003755EE7
:1052BC0001AE55AF56AC53AD54EF2DFDEE3CFC7426
:1052CC00028C068D071200398E558F569000B5E072
:1052DC0060099000B5E0C3943D4002804390001CEF
:1052EC00E0FEA3E0FF9000B5E08E048F05FF127086
:1052FC007574018C068D07120039900020EEF0A316
:10530C00EFF0900020E0F8A3E090001EC8F0A3C8D6
:10531C00F090001CE4F0A3F0C215E5B554FBF5B514
:10532C00A2A4B34002C21DA2A3B34002C21EA21C7F
:10533C00B34002C21CA218B34006A21A92198002F2
:10534C00B21990009DE06012E56D700EA218B3507A
:10535C0009A219301A01B3B34002800674059000FB
:10536C0054F0C218803AAE55AF56AC53AD54EF2D35
:10537C00FDEE3CFC74018C068D071200398E558FA6
:10538C0056E56DC39402500DAC53AD5474B8C39D27
:10539C00740B9C400280091246FF7406900054F076
:1053AC00E55EB43B127403900054F0D21C9000D212
:1053BC00E0B401031246FFAE57AF58AC53AD54EFF7
:1053CC002DFDEE3CFC8C578D58AE53AF54EFD39D56
:1053DC00EE9C4011900012E0FAA3E0FBEBC394E8C2
:1053EC00EA94034002800690001212709390001011
:1053FC00E0FEA3E0FFAC53AD54EF2DFDEE3CFC9072
:10540C000010ECF0A3EDF09000D2E0B40118AE5314
:10541C00AF547405127085740112003990000CEEB3
:10542C00F0A3EFF08011AE53AF547402127085905C
:10543C00000CEEF0A3EFF0C28E758D00758B00752D
:10544C006400755401755300D28EE55E240E75F020
:10545C000F84AFF07E00EF4E60030254EBE56D60FD
:10546C0013AE55AF56740F12708590000EEEF0A36C
:10547C00EFF0800F900010E0F8A3E090000EC8F061
:10548C00A3C8F090000EE0FEA3E0FFEF4E600B7C93
:10549C007C7D1A126F738E518F52900010E4F0A322
:1054AC00F0AE51AF527428BE00039F5010E5632F2D
:1054BC00FF50010E74011200398E518F52855263C8
:1054CC009000D9E0A851B8000DD395524008E55290
:1054DC00900053F080099000D9E014900053F090A4
:1054EC0000D0E0B40408900049E0655E6002800BD7
:1054FC00A219B34004D21B8002B21BE55E640B60A0
:10550C0005E55EB429099000C2E06003122C84907A
:10551C0000C7E0B40114900051E0655E6007900094
:10552C0052E0B55E03756F00801E900051E0655E21
:10553C006013900051E02414655E6009900051E006
:10554C002428B55E03756F00A20AB35006A209B3F6
:10555C00B3400302560790008EE0B4017390011023
:10556C00E0B40214121244900078E075F0BCA4FF71
:10557C00AEF08E5B8F5C8056E56775F00A84FF7E1B
:10558C0000900588120048E0F55A755900AE59AFE5
:10559C005A9000B3E012708574648E048F05FF126C
:1055AC0070758C5B8D5CE55C90004FF0AE59AF5A1A
:1055BC0090008CE012708574648E048F05FF12705D
:1055CC007574BC8C068D071270858E5B8F5C801792
:1055DC0090008CE075F0BCA4FFAEF08E5B8F5C90FD
:1055EC0000B3E090004FF0E561C394CC5006E55C4D
:1055FC00455B70028003124A74D20AE56DB4010651
:10560C00E55E6411600280097570009000557401AC
:10561C00F0E56D60030256BA9000D5E0600D900085
:10562C0077E0A851B800069552400280409000D512
:10563C00E0B4021F900046E0655E600F900047E00A
:10564C00655E6007900048E0B55E03757003756C8D
:10565C0000800CC201756C0090001AE4F0A3F0906D
:10566C000077E060067409900054F0804190004689
:10567C00E0655E600F900047E0655E600790004853
:10568C00E0B55E2A757000900046E0B55E069000AD
:10569C00557401F0900047E0B55E06740290005519
:1056AC00F0900048E0B55E067403900055F0A20738
:1056BC00B39205A207B330B601B350030257A175DC
:1056CC006E019000B5E0B43D13A207B34008E5B5F8
:1056DC004404F5B58006E5B554FBF5B5E5B54401D4
:1056EC00F5B5742B900072F0A2079205E55ED39489
:1056FC004A4014D209E55ED39485400B74049000A3
:10570C0054F0D21C755E469000DDE0B40107E56AEA
:10571C00C3944140028018E56AC394145008741372
:10572C00900054F08006740E900054F01246FF90D6
:10573C00005CE0FE900059E0C39E4009900059E0E7
:10574C00D39408400974FB900054F01246FF90006B
:10575C005AE0601590005AE0FE900058E06E600927
:10576C0074FC900054F01246FF90005BE0601590C2
:10577C00005BE0FE90005DE06E600974FE900054EA
:10578C00F01246FF90089FE0600690010DE0600269
:10579C008003120B97A21CB34006C296C295C2A0FE
:1057AC0090010DE0600CAE51AF527414BE00059F19
:1057BC0040028037900095E090699DF8282873800E
:1057CC002A8028A2A3B35005A21EB3400280051262
:1057DC004ABED21E8015A2A4B35005A21DB340022E
:0B57EC008005124ABED21D8002800022
:10699D000257CB0257CD0257CF0257E20257F502ED
:0269AD0057F79A
:1057F700A20CB3B35008900049E0655E60030259FC
:1058070065A202B35006A201B3B3400302595F90E9
:1058170000D0E0B404028003025923123CD8900858
:10582700F2E0B402028003025911A21BB340679051
:105837000121E0601F900018E0FEA3E0FF9001192E
:10584700E012708574C88E048F05FF1270758C5B2B
:105857008D5C800A900018E0F55BA3E0F55CAE5B19
:10586700AF5C745E12708574058E048F05FF12702D
:1058770075AE59AF5AED2FFFEC3EFE8E5B8F5C90F5
:105887000038E0FCA3E0FDEF2DFDEE3CFC8C5B8DCA
:105897005C123D588068900121E0D39403401F902B
:1058A7000018E0FEA3E0FF90011CE012708574C8A9
:1058B7008E048F05FF1270758C5B8D5C800A9000DB
:1058C70018E0F55BA3E0F55CAE5BAF5C745E12704D
:1058D7008574058E048F05FF127075AE59AF5AEDAA
:1058E7002FFFEC3EFE8E5B8F5C900038E0FCA3E060
:1058F700FDEF2DFDEE3CFC8C5B8D5C123D7990003D
:10590700EEE0B40103123D9A8010123D58123D7922
:105917009000EEE0B40103123D9A8039123CD81290
:105927003D589000D0E0B4030ED2929000EEE0B460
:105937000103123D9A801E9000EEE0B40206123D6C
:105947001A123D799000EEE0B40106A203B3B3400A
:10595700028002D29275A700C20CD20DD20EA20D00
:10596700B3B3500890004AE0655E6003025AE6A2AE
:1059770002B35006A201B3B34003025AE09000D02D
:10598700E0B404028003025A94123CD89008F2E073
:10599700B402028003025A82A21BB3406A9001211B
:1059A700E0D39401401F900018E0FEA3E0FF9001B0
:1059B7001AE012708574C88E048F05FF1270758CFB
:1059C7005B8D5C800A900018E0F55BA3E0F55CAEA8
:1059D7005BAF5C745E12708574058E048F05FF12D1
:1059E7007075AE59AF5AED2FFFEC3EFE8E5B8F5CA4
:1059F700900038E0FCA3E0FDEF2DFDEE3CFC8C5B56
:105A07008D5C123D638068900121E0D39404401FB0
:105A1700900018E0FEA3E0FF90011DE0127085746E
:105A2700C88E048F05FF1270758C5B8D5C800A90A1
:105A37000018E0F55BA3E0F55CAE5BAF5C745E124B
:105A4700708574058E048F05FF127075AE59AF5AB5
:105A5700ED2FFFEC3EFE8E5B8F5C900038E0FCA3E1
:105A6700E0FDEF2DFDEE3CFC8C5B8D5C123D8490E0
:105A770000EEE0B40103123D9A8010123D63123D1F
:105A8700849000EEE0B40103123D9A8049123CD89D
:105A9700123D639000EEE0C394025007A203B340A7
:105AA70002D2879000D0E0B4030ED2879000EEE0D8
:105AB700B40103123D9A801E9000EEE0B402061274
:105AC7003D1A123D849000EEE0B40106A203B3B381
:105AD70040028002D28775A700D20CC20DD20EA257
:105AE7000EB3B3500890004BE0655E6003025C673D
:105AF700A202B35006A201B3B34003025C61900057
:105B0700D0E0B404028003025C15123CD89008F27E
:105B1700E0B402028003025C03A21BB3406A900157
:105B270021E0D39402401F900018E0FEA3E0FF900D
:105B3700011BE012708574C88E048F05FF12707503
:105B47008C5B8D5C800A900018E0F55BA3E0F55C48
:105B5700AE5BAF5C745E12708574058E048F05FFB3
:105B6700127075AE59AF5AED2FFFEC3EFE8E5B8F6C
:105B77005C900038E0FCA3E0FDEF2DFDEE3CFC8CD3
:105B87005B8D5C123D6E8068900121E0D3940540E7
:105B97001F900018E0FEA3E0FF90011EE012708541
:105BA70074C88E048F05FF1270758C5B8D5C800A3C
:105BB700900018E0F55BA3E0F55CAE5BAF5C745E4C
:105BC70012708574058E048F05FF127075AE59AF7C
:105BD7005AED2FFFEC3EFE8E5B8F5C900038E0FCA9
:105BE700A3E0FDEF2DFDEE3CFC8C5B8D5C123D8F41
:105BF7009000EEE0B40103123D9A8010123D6E1240
:105C07003D8F9000EEE0B40103123D9A8049123CAB
:105C1700D8123D6E9000EEE0C394025007A203B382
:105C27004002D2909000D0E0B4030ED2909000EEE4
:105C3700E0B40103123D9A801E9000EEE0B4020624
:105C4700123D1A123D8F9000EEE0B40106A203B395
:105C5700B340028002D29075A700D20CD20DC20EBB
:0D5C6700E5709069AFF82828739000F5E013
:0369AF00025C7017
:105C74009069E2F82828731225CF80121225CF806C
:0E5C84000D12265980081227058003122705ED
:0F69E200025C7B025C80025C85025C8A025C8F37
:105C9200757001026178122831122948757002026A
:105CA2006178122CC8A204B340139000DAE075F0B8
:105CB2001DA4FFAEF0900014EEF0A3EFF090088860
:105CC200E0FEA3E0FF740A12708590000EE0FCA3D0
:105CD200E0FD74098F02FF1270758D078C038E042C
:105CE2008A058B06126F7390088CEEF0A3EFF074A6
:105CF200F0BE00039F500B74F090088CF8E4F0E8BB
:105D0200A3F0E536700375360190088CE0FEA3E03F
:105D1200FFE5362FFF50010E90088CEEF0A3EFF056
:0B5D2200757003A22E401A900055E09F
:0669B200025C98025CA4E7
:105D2D009069F1F8282873800D75700A80087570D8
:065D3D000B800375700CE1
:0C69F100025D34025D36025D3B025D4039
:105D43000261789006CFE060077401F508122DF622
:105D5300A230B3B35008900786E0642A600280093A
:105D6300E5B54402F5B5025E0D9000C3E0D394029D
:105D73004045900097E02403A851B8000495525081
:105D830009900099E0D395615002800ED202A226B9
:105D930040067408900054F0D226900097E0A85172
:105DA300B80005D39552500B900099E02403C39596
:105DB300615002C2028053900097E02403A851B8B7
:105DC300000495525010E55FC39560500990009907
:105DD300E0D395615002800ED202A22640067408D9
:105DE300900054F0D226900097E0A851B80005D354
:105DF30095525014E560240FC3955F400B900099B2
:105E0300E02403C395615002C202A2024002C226EB
:105E1300A230B3500DA202B35008900786E0642A63
:105E230060028006E5B554FDF5B59000DDE070072E
:105E3300E56AC3941440028002D2029000D2E0B417
:105E43000102D202A2024005757004800A75701027
:0E5E530090001AE4F0A3F00261789000C3E022
:0669B800025D46025E5D77
:105E61009069FDF828287312135A801212135A8070
:0E5E71000D12150D80081215C480031215C401
:0F69FD00025E68025E6D025E72025E77025E7C71
:105E7F009006D3E060077402F508122DF6757005D1
:105E8F0002617812171D7570069006D7E0600774CF
:105E9F0003F508122DF69006DBE060077404F50891
:105EAF00122DF602617890004FE06006A204B3B3A2
:105EBF004002800DE55ED39414500690004FE0141D
:105ECF00F01219A67570079006DFE060077405F5EC
:105EDF0008122DF69006E3E060077406F508122D00
:105EEF00F6026178900110E0B402031212CB121E79
:105EFF000E7570089006E7E060077407F508122D1D
:105F0F00F69006EBE060077408F508122DF60261B3
:105F1F0078121EF07570090261781222C8A20CB3B4
:105F2F005005A20DB340028006D20CD20DD20E75D1
:105F3F00701002617890003CE0C394465008C296FE
:105F4F00744690003CF090004CE0B4011DE53624FF
:105F5F0006F53690088CE0FEA3E0FF74062FFF5085
:105F6F00010E90088CEEF0A3EFF090004CE0B4021D
:105F7F001DE536240CF53690088CE0FEA3E0FF7487
:105F8F000C2FFF50010E90088CEEF0A3EFF085362A
:105F9F005A755900900046E0F573123EDEE55C90AD
:105FAF00003CF0900006E559F0A3E55AF0E5739038
:105FBF00003DF0C21090088CE0F559A3E0F55A901F
:105FCF000046E0F573123EDEE55C90003AF090007B
:105FDF0000E559F0A3E55AF0E57390003BF0C20FCE
:105FEF00E56DB4010575700B800375700302617860
:105FFF00900040E0C394465008C29574469000400C
:10600F00F090004DE0B4011DE5362406F5369008FA
:10601F008CE0FEA3E0FF74062FFF50010E90088C5A
:10602F00EEF0A3EFF090004DE0B4021DE536240C26
:10603F00F53690088CE0FEA3E0FF740C2FFF5001A3
:10604F000E90088CEEF0A3EFF085365A755900903C
:10605F000047E0F573123EDEE55C900040F09000E3
:10606F0008E559F0A3E55AF0E573900041F0C2122C
:10607F0090088CE0F559A3E0F55A900047E0F573CE
:10608F00123EDEE55C90003EF0900002E559F0A371
:10609F00E55AF0E57390003FF0C211E56DB40105CC
:1060AF0075700C8003757003026178900044E0C333
:1060BF0094465008C2A07446900044F090004EE001
:1060CF00B4011DE5362406F53690088CE0FEA3E0FA
:1060DF00FF74062FFF50010E90088CEEF0A3EFF027
:1060EF0090004EE0B4021DE536240CF53690088C76
:1060FF00E0FEA3E0FF740C2FFF50010E90088CEE12
:10610F00F0A3EFF085365A755900900048E0F5730B
:10611F00123EDEE55C900044F090000AE559F0A3D2
:10612F00E55AF0E573900045F0C21490088CE0F545
:10613F0059A3E0F55A900048E0F573123EDEE55C96
:10614F00900042F0900004E559F0A3E55AF0E57392
:10615F00900043F0C213E56DB40103756D007570C7
:09616F0003800680048002800018
:1069BE00025E92025EB5025EF3025F20025F290262
:1069CE005F44025FFF0260BA02617202617402618B
:0469DE007602617864
:1061780090003AE0B55E02800302621AA20F4072F4
:10618800900000E0FEA3E0FFEF4E6021AE55AF5651
:10619800900000E0FCA3E0FD12000374068E048F5B
:1061A80005FF127075900000ECF0A3EDF090003B35
:1061B800E0601A900000E0FEA3E0FFAC55AD56EF9A
:1061C8002DFDEE3CFC900000ECF0A3EDF090003BC0
:1061D800E0D39401401A900000E0FEA3E0FFAC5524
:1061E800AD56EF2DFDEE3CFC900000ECF0A3EDF079
:1061F800D20FAE53AF54900000E0FCA3E0FDEFC314
:106208009DEE9C400D124B05D296C20F74C89000AB
:106218003AF0A20FB3B3500790003AE0B55E02809F
:106228000D124B05D29674C890003AF0C20F900038
:106238003CE0B55E0280030262D5A2104072900075
:1062480006E0FEA3E0FFEF4E6021AE55AF5690008A
:1062580006E0FCA3E0FD12000374068E048F05FF20
:10626800127075900006ECF0A3EDF090003DE06030
:106278001A900006E0FEA3E0FFAC55AD56EF2DFDE9
:10628800EE3CFC900006ECF0A3EDF090003DE0D36E
:106298009401401A900006E0FEA3E0FFAC55AD560D
:1062A800EF2DFDEE3CFC900006ECF0A3EDF0D210D3
:1062B800AE53AF54900006E0FCA3E0FDEFC39DEEA3
:1062C8009C400AC296744690003CF0C210A210B3DB
:1062D800B3500790003CE0B55E02800AC29674464F
:1062E80090003CF0C21090003EE0B55E02800302D0
:1062F8006390A2114072900002E0FEA3E0FFEF4E0F
:106308006021AE55AF56900002E0FCA3E0FD1200FC
:106318000374068E048F05FF127075900002ECF06E
:10632800A3EDF090003FE0601A900002E0FEA3E0C9
:10633800FFAC55AD56EF2DFDEE3CFC900002ECF0A5
:10634800A3EDF090003FE0D39401401A900002E0E2
:10635800FEA3E0FFAC55AD56EF2DFDEE3CFC9000E2
:1063680002ECF0A3EDF0D211AE53AF54900002E06E
:10637800FCA3E0FDEFC39DEE9C400D124B05D295AA
:10638800C21174C890003EF0A211B3B35007900038
:106398003EE0B55E02800D124B05D29574C89000A0
:1063A8003EF0C211900040E0B55E02800302644BEB
:1063B800A2124072900008E0FEA3E0FFEF4E6021B9
:1063C800AE55AF56900008E0FCA3E0FD1200037440
:1063D800068E048F05FF127075900008ECF0A3ED8F
:1063E800F0900041E0601A900008E0FEA3E0FFACE6
:1063F80055AD56EF2DFDEE3CFC900008ECF0A3EDFA
:10640800F0900041E0D39401401A900008E0FEA308
:10641800E0FFAC55AD56EF2DFDEE3CFC900008ECCE
:10642800F0A3EDF0D212AE53AF54900008E0FCA3F5
:10643800E0FDEFC39DEE9C400AC295744690004073
:10644800F0C212A212B3B35007900040E0B55E024A
:10645800800AC2957446900040F0C212900042E053
:10646800B55E028003026506A2134072900004E044
:10647800FEA3E0FFEF4E6021AE55AF56900004E05A
:10648800FCA3E0FD12000374068E048F05FF127052
:1064980075900004ECF0A3EDF0900043E0601A90D2
:1064A8000004E0FEA3E0FFAC55AD56EF2DFDEE3C39
:1064B800FC900004ECF0A3EDF0900043E0D39401CD
:1064C800401A900004E0FEA3E0FFAC55AD56EF2D56
:1064D800FDEE3CFC900004ECF0A3EDF0D213AE53BB
:1064E800AF54900004E0FCA3E0FDEFC39DEE9C4098
:1064F8000D124B05D2A0C21374C8900042F0A2132B
:10650800B3B35007900042E0B55E02800D124B0510
:10651800D2A074C8900042F0C213900044E0B55E67
:106528000280030265C1A214407290000AE0FEA333
:10653800E0FFEF4E6021AE55AF5690000AE0FCA395
:10654800E0FD12000374068E048F05FF127075902B
:10655800000AECF0A3EDF0900045E0601A90000A04
:10656800E0FEA3E0FFAC55AD56EF2DFDEE3CFC90F0
:10657800000AECF0A3EDF0900045E0D39401401A36
:1065880090000AE0FEA3E0FFAC55AD56EF2DFDEEFE
:106598003CFC90000AECF0A3EDF0D214AE53AF54DB
:1065A80090000AE0FCA3E0FDEFC39DEE9C400AC208
:1065B800A07446900044F0C214A214B3B3500790DC
:1065C8000044E0B55E02800AC2A07446900044F020
:1065D800C2149000E0E0B4020280030266F6900064
:1065E80074E0D395665064900074E0F4042566FE68
:1065F8009000E3E08E00F5F0E884FF7E008F73EFF3
:10660800C39410500CEF8573F0A4FDACF08D73802B
:10661800037573FF900074E0D39573400B9000747A
:10662800E0C39573F57180037571009000FEE0D3A7
:10663800957140069000FEE0F5719000FFE0C3956B
:106648007150069000FFE0F5718071900074E0C30E
:106658009566FE9000E3E08E00F5F0E884FF7E008A
:106668008F73EFC39410500CEF8573F0A4FDACF05A
:106678008D7380037573FF85735A75590090007484
:10668800E0255AFFAE5950010E8E598F5A74FFBE3D
:106698000009D39F4005855A7180037571FF9000EA
:1066A800FEE0D3957140069000FEE0F5719000FF82
:1066B800E0C3957150069000FFE0F571A204B3B3F2
:1066C800500D900075E0FE9000EBE0D39E500280E4
:1066D8000A7407900054F0C297801375A710E5CD8F
:1066E800C395714004C2978002D29775A700A2048F
:1066F800B350030267BA900105E0A851B8000495A9
:10670800525017900104E0A851B8000ED39552409A
:1067180009900106E0D395614002802375A710E532
:10672800CDC394805008E5B54480F5B58006E5B53D
:10673800547FF5B5E5B554BFF5B575A7008021754B
:10674800A710E5CDC394805008E5B54440F5B58061
:1067580006E5B554BFF5B5E5B5547FF5B575A700A1
:10676800900108E0A851B80004955250179001070D
:10677800E0A851B8000ED395524009900109E0D322
:1067880095614002801775A710E5CDC39480500429
:10679800D2A18002C2A1C2A275A700801575A71058
:1067A800E5CDC394805004D2A28002C2A2C2A175D2
:1067B800A700E56FC39413501DE56F75F00284AF11
:1067C800F07E00EF4E7005123290800AA2EDB340C1
:1067D80005C2ED123290AE53AF547410C39F7427A4
:1067E8009E400C900073E0C3945A4003026958A27B
:1067F80009B340091246FF7406900054F0A20BB387
:10680800500EE561D394334007E561C394CC400250
:106818008041900110E0B40214121244900078E014
:1068280075F05EA4FFAEF08E5B8F5C800F90008CDD
:10683800E075F05EA4FFAEF08E5B8F5CE55C455BB7
:106848006011E5B54401F5B5742B900072F0124A59
:1068580074D20B900073E0D394014007E561C394B0
:106868001A40028002C20B9006CFE060077401F55F
:1068780008122DF69006D3E060077402F508122D71
:10688800F69006D7E060077403F508122DF6900617
:10689800DBE060077404F508122DF69006DFE0606F
:1068A800077405F508122DF69006E3E060077406F4
:1068B800F508122DF69006E7E060077407F5081250
:1068C8002DF69006EBE060077408F508122DF69097
:1068D8000073E0C3945A5010E56FB4130990007325
:1068E800E004F0756F00803FE56FB41303756F0027
:1068F800C28E758D00758B007564007554017553D3
:1069080000D28E900072E0C394415008900072E06B
:1069180004F080067441900072F0900072E0B44177
:1069280006E5B554FEF5B5900073E0D39401400731
:10693800E56AC3944140028006740E900054F090BA
:10694800089FE0600690010DE060028003120B973B
:03695800025014D6
:106A0C000000010001400160018001A001C001E013
:106A1C0002000300039603B603D603F4040005003A
:106A2C000512052405360548055A056C057E0590AA
:106A3C0005A805C005DE0600061406280646066EE7
:106A4C0006AE05CF06EE00FF013F015F017F019FFF
:106A5C0001BF01DF01FF02FF039503B503D503F36B
:106A6C0003FF04FF05110523053505470559056B83
:106A7C00057D058F05A705BF05CE05F10613062775
:106A8C000645066D06AD06ED05DD06FF0FAA0FA542
:106A9C000F9F0F9A0F940F8D0F870F800F780F7128
:106AAC000F680F600F570F4E0F450F3B0F300F2520
:106ABC000F1A0F0E0F020EF50EE80EDB0ECC0EBEEB
:106ACC000EAE0E9F0E8E0E7D0E6C0E5A0E470E34B1
:106ADC000E200E0C0DF70DE20DCB0DB50D9D0D8599
:106AEC000D6D0D540D3A0D200D050CE90CCE0CB1AD
:106AFC000C940C760C580C3A0C1B0BFB0BDB0BBBE5
:106B0C000B9A0B790B570B350B130AF10ACE0AAB08
:106B1C000A870A640A400A1C09F809D409B0098CCE
:106B2C0009670943091F08FB08D608B2088E086AD2
:106B3C000846082307FF07DC07B9079607730751B8
:106B4C00072F070D06EC06CA06AA06890669064930
:106B5C00062A060A05EC05CD05B005920575055803
:106B6C00053C0520050504EA04CF04B5049C048209
:106B7C000469045104390422040B03F403DE03C832
:106B8C0003B2039D038903750361034D033B032883
:106B9C000316030402F202E102D102C002B002A009
:106BAC00029102820273026502570249023C022FD3
:106BBC0002220216020901FD01F201E601DB01D0FD
:106BCC0001C601BB01B101A7019D0194018B01829A
:106BDC0001790170016801600158015001480141BF
:106BEC0001390132012B0125011E01180111010B84
:106BFC00010500FF00FA0FA60FA00F990F920F8B43
:106C0C000F840F7C0F740F6B0F620F580F4E0F43D6
:106C1C000F380F2C0F1F0F120F050EF70EE80ED8A2
:106C2C000EC80EB70EA50E930E800E6C0E580E42AB
:106C3C000E2C0E150DFD0DE40DCB0DB10D950D7932
:106C4C000D5D0D3F0D200D010CE10CC00C9E0C7C5C
:106C5C000C590C350C100BEA0BC40B9E0B760B4F1E
:106C6C000B260AFD0AD40AAA0A800A550A2A09FF29
:106C7C0009D409A8097C0950092508F908CD08A1EF
:106C8C000875084A081E07F307C8079D07730749CC
:106C9C00072006F706CE06A6067E06570630060A1D
:106CAC0005E405BF059B057705540532051004EF77
:106CBC0004CE04AE048F047104530435041903FD8F
:106CCC0003E203C703AD0394037B0363034B033459
:106CDC00031E030802F302DE02CA02B602A30291EB
:106CEC00027F026D025C024C023C022C021D020E61
:106CFC00020001F201E401D701CA01BE01B101A6F3
:106D0C00019A018F0185017A01700166015D0153C1
:106D1C00014A0141013901310129012101190112F5
:106D2C00010B010400FD00F700F000EA00E400DEB6
:106D3C0000D900D300CE00C900C400BF00BA00B512
:106D4C0000B100AD00A800A400A0009C0099009523
:106D5C000091008E008A008700840081007E007BF9
:10009E0075B50075840175A70075FFA075EF069004
:1000AE000050E4F075C91075A70F75A1C775A700AC
:1000BE0075D90075CE0C75A70F75F1FE75F2FF752B
:1000CE00F30775F47875A4BA75A5FF75A60775AE16
:1000DE000075AFFF75D48175D5FF75D6FF75D7FF47
:1000EE0075A70075A20175A14775F8092275E60876
:1000FE0075E71075BC0175BE0475BD6C75BE0775D0
:10010E00BDA075BE0875BD0175BC0075BB1875BC6C
:10011E002075BA0875E88075D11375A70F75E105BE
:10012E0075E20075C7401246FF759700759780748B
:10013E000A1270657597C0E5975420700280F875A5
:10014E008F0275A700D2AF75980075A90C75A70F11
:10015E0075AB4375ADFB75AC1E75A71075C91875DB
:10016E00CA0075CB0075C80475A700758912758E07
:10017E0004758C00758A00C2A9D28C758D00758BA2
:10018E0000D2ABD28E75B62075D944C2992290009A
:10019E008AE090089EF0900095E090089FF0900005
:1001AE0096E09008A0F09000B5E09008A1F09000C5
:1001BE00C2E09008A2F09000D0E09008A3F090006A
:1001CE00DEE09008A4F09000E0E09008A5F090002A
:1001DE00EEE09008A6F09000FBE09008A7F09000EB
:1001EE00FCE09008A8F090010EE09008A9F09001B4
:1001FE0026E09008ABF0900174E09008ACF090010E
:10020E0075E09008ADF0900176E09008AEF09001A8
:10021E000DE09008AFF09000F7E09008B0F090007D
:10022E00AEE09008B1F09000AFE09008B2F0900010
:10023E00A9E09008B3F09000AAE09008B4F0900105
:10024E0013E09008B5F0900114E09008B6F090011C
:10025E0015E09008B7F0900116E09008B8F0900104
:10026E0017E09008B9F09006CEE09008BAF090062C
:10027E00D2E09008BBF09006D6E09008BCF0900655
:10028E00DAE09008BDF09006DEE09008BEF0900631
:10029E00E2E09008BFF09006E6E09008C0F090060D
:1002AE00EAE09008C1F09006EEE09008C2F09006E9
:1002BE00F2E09008C3F0900776E09008C4F0900743
:1002CE0077E09008C5F0900778E09008C6F09007A8
:1002DE0079E09008C7F090077AE09008C8F0900790
:1002EE007BE09008C9F090077CE09008CAF0900778
:1002FE007DE09008CBF090077EE09008CCF0900760
:10030E007FE09008CDF0900780E09008CEF0900747
:10031E0081E09008CFF0900782E09008D0F090072F
:10032E0083E09008D1F0900784E09008D2F0900717
:10033E0085E09008D3F0900786E09008D4F0900105
:10034E0018E09008D5F0900119E09008D6F09001D1
:10035E001AE09008D7F090011BE09008D8F09001B9
:10036E001CE09008D9F090011DE09008DAF09001A1
:10037E001EE09008DBF090011FE09008DCF0900189
:10038E0020E09008DDF0900121E09008DEF0229050
:10039E00089EE090008AF090089FE0900095F09003
:1003AE0008A0E0900096F09008A1E09000B5F090C3
:1003BE0008A2E09000C2F09008A3E09000D0F09068
:1003CE0008A4E09000DEF09008A5E09000E0F09028
:1003DE0008A6E09000EEF09008A7E09000FBF090E9
:1003EE0008A8E09000FCF09008A9E090010EF090B3
:1003FE0008ABE0900126F09008AFE090010DF09070
:10040E0008B0E09000F7F09008B1E09000AEF090E8
:10041E0008B2E09000AFF09008B3E09000A9F09021
:10042E0008B4E09000AAF09008B5E0900113F090A7
:10043E0008B6E0900114F09008B7E0900115F09026
:10044E0008B8E0900116F09008B9E0900117F0900E
:10045E0008BAE09006CEF09008BBE09006D2F0907D
:10046E0008BCE09006D6F09008BDE09006DAF09059
:10047E0008BEE09006DEF09008BFE09006E2F09035
:10048E0008C0E09006E6F09008C1E09006EAF09011
:10049E0008C2E09006EEF09008C3E09006F2F090ED
:1004AE0008C4E0900776F09008C5E0900777F090CA
:1004BE0008C6E0900778F09008C7E0900779F090B2
:1004CE0008C8E090077AF09008C9E090077BF0909A
:1004DE0008CAE090077CF09008CBE090077DF09082
:1004EE0008CCE090077EF09008CDE090077FF0906A
:1004FE0008CEE0900780F09008CFE0900781F09052
:10050E0008D0E0900782F09008D1E0900783F09039
:10051E0008D2E0900784F09008D3E0900785F09021
:10052E0008D4E0900786F09008D5E0900118F0907E
:10053E0008D6E0900119F09008D7E090011AF090DB
:10054E0008D8E090011BF09008D9E090011CF090C3
:10055E0008DAE090011DF09008DBE090011EF090AB
:10056E0008DCE090011FF09008DDE0900120F09093
:10057E0008DEE0900121F022754700900896E4F025
:10058E00A3F0753100753000754D00754E00C22A0E
:10059E00D22B90089FE06002D21F74FE900898F84C
:1005AE00E4F0E8A3F074FE90089CF8E4F0E8A3F001
:1005BE0074FE90089AF8E4F0E8A3F0745A9008F0EC
:1005CE00F0745A9008F1F0D22CC228C22EC22DC25D
:1005DE0029C230C23622750B00750A00AE0AAF0B67
:1005EE00AC08AD09EDC39FEC9E401674FF1270650A
:1005FE0075CF01780B740126F6500418E436F650C8
:10060E00DB22C2AF75D904758F0375B7A575B7F127
:10061E0090F800E4F0758F0175B7A575B7F1E52771
:10062E0090F800F075B7A575B7F190F801E4F07584
:10063E00B7A575B7F19008E4E090F802F075B7A58C
:10064E0075B7F19008E8E090F803F075B7A575B7A7
:10065E00F19008E5E090F804F075B7A575B7F19044
:10066E0008E6E090F805F075B7A575B7F19008E7C4
:10067E00E090F806F075B7A575B7F19008E9E0902F
:10068E00F807F0758F0075D944D2AF22900050E074
:10069E00B4AB61C2AF75D90475B62275F522758FEC
:1006AE000375B7A575B7F1740090F600F0758F015C
:1006BE00755A00755900AE59AF5A7445BE00279F42
:1006CE00402475B7A575B7F190089E120048E0FC5E
:1006DE0090F600120048ECF0785A740126F6500499
:1006EE0018E436F650D0758F0075F51175B6207575
:1006FE00D944D2AF22C2AF75F52275D904755A000E
:10070E00755900AE59AF5A7445BE00229F401F90D6
:10071E00F600120048E493FC90089E120048ECF09C
:10072E00785A740126F6500418E436F650D575D969
:10073E004475F511D2AF22900050E0B4AA028003A6
:10074E00020882C2AF75D90475B62275F522758F6F
:10075E000375B7A575B7F1740090F400F075B7A5E1
:10076E0075B7F1740090F200F075B7A575B7F17416
:10077E000090F000F075B7A575B7F1740090EE001B
:10078E00F0758F01755A00755900AE59AF5A74FF46
:10079E00C39F74019E402475B7A575B7F19000886C
:1007AE00120048E0FC90F400120048ECF0785A7405
:1007BE000126F6500418E436F650CF755A007559D6
:1007CE0000AE59AF5A74FFC39F74019E402475B793
:1007DE00A575B7F1900288120048E0FC90F2001265
:1007EE000048ECF0785A740126F6500418E436F6F8
:1007FE0050CF755A00755900AE59AF5A74FFC39F4A
:10080E0074019E402475B7A575B7F1900488120047
:10081E0048E0FC90F000120048ECF0785A74012683
:10082E00F6500418E436F650CF755A00755900AEDE
:10083E0059AF5A74FFC39F74019E402475B7A575B6
:10084E00B7F1900688120048E0FC90EE00120048C6
:10085E00ECF0785A740126F6500418E436F650CFB0
:10086E00758F0075F51175B62075D944D2AF743AEF
:10087E00900788F022900050E0B4AA02800302098B
:10088E00C0C2AF75D90475B62275F522758F037582
:10089E00B7A575B7F1740090EC00F075B7A575B7F4
:1008AE00F1740090EA00F075B7A575B7F174009079
:1008BE00E800F075B7A575B7F1740090E600F07515
:1008CE008F01755A00755900AE59AF5A74FFC39F08
:1008DE0074019E402475B7A575B7F190008812007B
:1008EE0048E0FC90EC00120048ECF0785A740126B7
:1008FE00F6500418E436F650CF755A00755900AE0E
:10090E0059AF5A74FFC39F74019E402475B7A575E5
:10091E00B7F1900288120048E0FC90EA00120048FD
:10092E00ECF0785A740126F6500418E436F650CFDF
:10093E00755A00755900AE59AF5A74FFC39F7401B2
:10094E009E402475B7A575B7F1900488120048E053
:10095E00FC90E800120048ECF0785A740126F6502C
:10096E000418E436F650CF755A00755900AE59AFDB
:10097E005A74FFC39F74019E402475B7A575B7F1D5
:10098E00900688120048E0FC90E600120048ECF059
:10099E00785A740126F6500418E436F650CF758F47
:1009AE000075F51175B62075D944D2AF743A90071B
:1009BE0088F022C2AF75D90475F522755A007559A3
:1009CE0000AE59AF5A74FFC39F74019E401F90F43E
:1009DE0000120048E493FC900088120048ECF07876
:1009EE005A740126F6500418E436F650D4755A009F
:1009FE00755900AE59AF5A74FFC39F74019E401FC4
:100A0E0090F200120048E493FC900288120048EC29
:100A1E00F0785A740126F6500418E436F650D47560
:100A2E005A00755900AE59AF5A74FFC39F74019E98
:100A3E00401F90F000120048E493FC9004881200CE
:100A4E0048ECF0785A740126F6500418E436F65045
:100A5E00D4755A00755900AE59AF5A74FFC39F74BE
:100A6E00019E401F90EE00120048E493FC90068811
:100A7E00120048ECF0785A740126F6500418E43649
:100A8E00F650D475F51175D944D2AF74019000D1DA
:100A9E00F0743A900788F09008F77401F022C2AF14
:100AAE0075D90475F522755A00755900AE59AF5AAD
:100ABE0074FFC39F74019E401F90EC00120048E427
:100ACE0093FC900088120048ECF0785A740126F6D8
:100ADE00500418E436F650D4755A00755900AE59C4
:100AEE00AF5A74FFC39F74019E401F90EA0012001C
:100AFE0048E493FC900288120048ECF0785A740196
:100B0E0026F6500418E436F650D4755A007559007E
:100B1E00AE59AF5A74FFC39F74019E401F90E800F8
:100B2E00120048E493FC900488120048ECF0785AC6
:100B3E00740126F6500418E436F650D4755A007532
:100B4E005900AE59AF5A74FFC39F74019E401F9057
:100B5E00E600120048E493FC900688120048ECF080
:100B6E00785A740126F6500418E436F650D475F50A
:100B7E001175D944D2AF74029000D1F0743A900737
:100B8E0088F074029008F7F02274019000D1F09072
:100B9E00089FE0903C1EF828287380188016A2A3A8
:100BAE00400674029000D1F0800AA2A4400674029E
:040BBE009000D1F0E2
:0C3C1E00020BA8020BAA020BAC020BB8B0
:100BC2009000D1E0B40105A234B34002801AD234BD
:100BD2001246FF1209C174019000D1F012039D1256
:100BE2003E1E741B900054F09000D1E0B40206A2A5
:100BF20034B3B34002801AC2341246FF120AAC74F4
:100C0200029000D1F012039D123E1E741B900054FC
:100C1200F022E54E64046006E59964FF60028031CB
:100C2200A22A4004D22A8027E54E600874E6254EA7
:100C3200900054F0E54D600874F0254D900054F09A
:100C4200E54EB4010280FE754E00754D00C22A8049
:100C520002C22AE54E903C2AF8282873754E00E518
:100C620099B4FF03754D01E599B4FE03754D02E594
:100C720099B4FD03754D03E599B4FC03754D04E584
:100C820099B4FA03754D05E599B4FB06754E011248
:100C920046FFE599B4F906754E041246FFE599B48C
:100CA200F7331246FFC29C74AB900050F012069AC2
:100CB20074AA900050F09008F7E0B40105120745BD
:100CC2008003120883900050E4F0D29C754E0075A8
:100CD2004D007599F7E599D394E54007E599C394DA
:100CE200F04002801685994F754E027E017F00E525
:100CF2004FC394E61270858E328F33900896E4F0DB
:100D0200A3F0E599D394C24007E599C394E6400263
:100D1200802885994F754E0374E5C3954FF5337559
:100D22003200AE32AF33906A0C127054E493F8740E
:100D32000193900896C8F0A3C8F0D2990210A2902D
:100D420008ABE0700AA220B35005A221B340028092
:100D52005C900896E0FEA3E0FF74FFBE00039F5084
:100D620009EFC39446EE9406402B900896E0FEA34A
:100D7200E0FFEFD3946DEE94064009EFC394EEEEDC
:100D820094064011900896E0FEA3E0FFEFD394FF93
:100D9200EE94064013900896E0FEA3E0FF900088D0
:100DA200120048E599F080038599748011900896A5
:100DB200E0FEA3E0FF900088120048E599F0900859
:100DC20096127093900896E0FEA3E0FFEFB401063E
:100DD200EEB407028003020E9B900788E0B43C0247
:100DE2008003020E9BA220B35005A221B3400280D1
:100DF20055C29C12039D900095E09008F6F0123FB8
:100E020075900174E09008ACF0900175E09008AD27
:100E1200F0900176E09008AEF074AB900050F012C2
:100E2200069A74AA900050F09008F7E0B4010512F7
:100E3200074580031208839008F7E09000D1F090F4
:100E42000050E4F08048C29C12019C74009008ACEF
:100E5200F074009008ADF074009008AEF090009528
:100E6200E09008F6F0123F7574AB900050F0120655
:100E72009A74AA900050F0120745120883D29C750A
:100E820099FB7464F5097508001205E480FED29C92
:100E9200754E00754D007599FB0210A2900896E000
:100EA200FEA3E0FFEF4E7006859931753000900881
:100EB20096E0FEA3E0FF74016F4E701BAC30AD31C3
:100EC200AA32AB33ED2BFBEC3AFA8A068B07900081
:100ED20088120048E599F09008961270939008964F
:100EE200E0FEA3E0FF74026F4E7021AC30AD3174AE
:100EF200566D4C7006E54F64E6600280031246FFB1
:100F0200123F75854F99754E00754D000210A290E3
:100F12000896E0FEA3E0FF900088120048E599F0F1
:100F2200900896127093900896E0FEA3E0FFAC3210
:100F3200AD338F028E038C068D07906A5212705465
:100F4200E493F9740193FEEAD39EEB994009854F2D
:100F520099754E00754D000210A2900896E0FEA30E
:100F6200E0FF900088120048E599F0900896127010
:100F720093900896E0FEA3E0FFEFB40006EEB40102
:100F82000280030210A2900066E0D394C7400B9047
:100F92000066E0C394C8F550801A900066E0D394CE
:100FA20063400B900066E0C39464F55080069000A5
:100FB20066E0F550E55075F002A4FFAEF08F73EFD6
:100FC2009000881270B6EFFCE0FDEC90008B12707E
:100FD200B6EDFCE0FDEC2DB5500280030210930F3C
:100FE200EF9000881270B6E573FFE0FCEF90008C82
:100FF2001270B6ECFFE0FCEFC39CB5500280030216
:101002001093E57390008A1270B6E573FFE0FCEF6F
:1010120090008D1270B6ECFFE0FCEF2CB55072E53B
:101022007390008E1270B6E0C395509008E4F0E51C
:101032007390008F1270B6E0C395509008E5F0E50A
:10104200739000921270B6E0C395509008E6F0E5F6
:10105200739000931270B6E0C395509008E7F0E5E4
:10106200739000941270B6E0C395509008E8F0E5D2
:10107200739000951270B6E0C395509008E9F01293
:1010820006107599F97464F5097508001205E48073
:10109200FE7599FF7464F5097508001205E480FE77
:0F3C2A00020C5E020D41020E9E020F11020F5C92
:1010A20022E54D903C39F828287302118790089662
:1010B200E0FEA3E0FF900056120048E0F599900888
:1010C20096127093900896E0FEA3E0FF741C6F4E98
:1010D2007003754D00021187856E99021187900881
:1010E20096E0FEA3E0FF900088120048E0F599EF39
:1010F200B40107EEB40703754D0090089612709381
:07110200021187900897E03D
:0F3C39000210AC0210AF0210DA0210E002110507
:10110900903CABF82828738552998067855F998050
:1011190062856199805D8565998058856799805355
:10112900856899804E8569998049856A9980449036
:10113900001BE0F599803CA22BB340077599FAC2D0
:101149002B8017A21FB3400575990F800B9000548F
:10115900E0F599900054E4F0C21F8017856B9980DF
:1011690012856699800D856C9980087599FC8003B4
:03117900754D00B1
:103CAB0002111002111502111A02111F0211240226
:103CBB00112902112E021133021138021140021187
:0D3CCB006502116A02116F02117402117975
:0B117C009008961270938003123E79D9
:033C4800021184E2
:1011870022E537255AFFAE5950010E90008812000C
:1011970048E0F538E537255AFFAE5950010E0FBF25
:1011A70000010E900088120048E0F539853F3BE5C5
:1011B70038B539058538378041E539D39538401D2D
:1011C700E539C39538853AF0A4FFAEF0E53B8E04C8
:1011D7008F05FF127075ED2538F537801DE538C38B
:1011E7009539853AF0A4FFAEF0E53B8E048F05FFF5
:1011F700127075EDF4042538F53722E539D39538A3
:10120700401DE539C39538853AF0A4FFAEF0E53BBC
:101217008E048F05FF127075ED2538F537801DE5B3
:1012270038C39539853AF0A4FFAEF0E53B8E048FBD
:1012370005FF127075EDF4042538F5372290008EFE
:10124700E0B4017FE56775F00A84FF7E008F37E51C
:101257006775F00A84ADF07C008D3A753F0A7559C1
:1012670005755A24E537C394115005121188800675
:101277009005BDE0F537E537C394F05008E53790A2
:101287000078F0800674EF900078F0E56775F00A53
:1012970084FF7E008F37E56775F00A84ADF07C0028
:1012A7008D3A753F0A755905755A5AE537C3941132
:1012B700500512118880069005F3E0F537E5379061
:1012C700004FF02290008EE0B40102800302135910
:1012D700E56775F00A84FF7E008F37E56775F00ACA
:1012E70084ADF07C008D3A753F0A755905755A36FD
:1012F700E537C39411500512118880069005CFE099
:10130700F537E537C394F0500585374B8003754BA8
:10131700EFE56775F00A84FF7E008F37E56775F0A4
:101327000A84ADF07C008D3A753F0A755905755AE8
:1013370048E537C39411500512118880069005E1DE
:10134700E0F537E537C394F0500585374C800375D2
:101357004CEF22E55F75F00484FF7E008F37E55F71
:1013670075F00484ADF07C008D3A753F0475590122
:10137700755A00E537C3943F5005121188800690CF
:1013870001C7E0F537E537900890F8E4F0E8A3F0F7
:10139700900053E075F020A4FFAEF09000D9E08EE6
:1013A700048F05FF1270758D379000C1E0D3955FEC
:1013B70050030214659000E5E0D3955F4010ED906F
:1013C70001C81270B6E0F52B752A0002146290006E
:1013D700B0E0D3955F4043E5379001C81270B6E09F
:1013E700F538E5379001E81270B6E0F5399000E579
:1013F700E0F404255FF53A9000B0E0FE9000E5E0E8
:10140700F4042EF53BE538B53905853837800312E6
:10141700120285372B752A008041E5379001E812C3
:1014270070B6E0F538E5379002081270B6E0F53986
:101437009000B0E0F404255FF53A9000C1E0FE901B
:1014470000B0E0F4042EF53BE538B53905853837AB
:10145700800312120285372B752A0002150C9000A3
:10146700E8E0D3955F5011E5379002481270B6E077
:10147700F52B752A0002150C9000B1E0D3955F504B
:1014870043E5379002281270B6E0F538E537900249
:10149700481270B6E0F5399000B1E0F404255FF525
:1014A7003A9000E8E0FE9000B1E0F4042EF53BE549
:1014B70038B53905853837800312120285372B7501
:1014C7002A008041E5379002081270B6E0F538E54A
:1014D700379002281270B6E0F5399000C1E0F404A5
:1014E700255FF53A9000B1E0FE9000C1E0F4042ECC
:1014F700F53BE538B5390585383780031212028583
:10150700372B752A00229000F9E0F53C753F1175DD
:101517005902755A00AE51AF52E53C75F00FA4FD64
:10152700ACF0EDD39FEC9E4021E53C8E048F05FF88
:10153700127075ED75F010A4FFAEF0E55F75F01150
:1015470084FD7C00ED2FF53D800EE55F75F011847D
:10155700FF7E00EF24F0F53D853D37E55F75F0111F
:1015670084AFF07E008F3A12118885373EAE51AFB7
:10157700529000F9E075F00FA4FDACF0EDD39FECAD
:101587009E4028755902755A10853D371211888576
:101597003E38853739AE51AF52E53C8E048F05FF93
:1015A7001270A08D3A853C3B121202E537900890E5
:1015B700F8E4F0E8A3F0752B64752A00229000F98F
:1015C700E0F53C753F11755902755A00AE51AF529F
:1015D700E53C75F00FA4FDACF0EDD39FEC9E4021E8
:1015E700E53C8E048F05FF127075ED75F010A4FFB2
:1015F700AEF0E56175F01184FD7C00ED2FF53D80BF
:101607000EE56175F01184FF7E00EF24F0F53D854E
:101617003D37E56175F01184AFF07E008F3A121106
:101627008885373EAE51AF529000F9E075F00FA4B0
:10163700FDACF0EDD39FEC9E4028755902755A100A
:10164700853D37121188853E38853739AE51AF52FF
:10165700E53C8E048F05FF1270A08D3A853C3B1246
:101667001202E537900890F8E4F0E8A3F0E56B6024
:1016770017E56BC394FE50109000EDE0B40209909B
:1016870000DBE0D3940B5002801F900890E0FEA38C
:10169700E0FFE56B12708574E78E048F05FF12700B
:1016A70075900890ECF0A3EDF09000C3E0B4045FF0
:1016B700E55F75F00484FF7E008F37E55F75F00402
:1016C70084ADF07C008D3A753F04755901755A0059
:1016D700E537C3943F500512118880069001C7E093
:1016E700F537900890E0FEA3E0FFE53712708574A8
:1016F700328E048F05FF127075900890E0FEA3E00C
:10170700FFEF2DFDEE3CFC900890ECF0A3EDF0759B
:101717002B64752A002290008EE0B40146E56775B8
:10172700F00A84FF7E008F37E56775F00A84ADF015
:101737007C008D3A753F0A755905755A00E537C320
:10174700941150051211888006900599E0F537AE7F
:101757002AAF2BE5372FFF50010E74641270C88E25
:101767002A8F2B90008FE0B40146E56875F00A8454
:10177700FF7E008F37E56875F00A84ADF07C008D39
:101787003A753F0A755905755A6CE537C394115078
:10179700051211888006900605E0F537AE2AAF2BB3
:1017A700E5372FFF50010E74641270C88E2A8F2BF5
:1017B70090009EE0B40249E56AC3944175F0058440
:1017C700FF7E008F37E56A75F00584ADF07C008DEC
:1017D7003A753F05755906755A00E537C394135096
:1017E70005121188800690069BE0F537AE2AAF2BCD
:1017F700E5372FFF50010E74641270C88E2A8F2BA5
:101807009000E0E0B4020280030218BCE55F75F0C7
:101817001584FF7E008F37E55F75F01584ADF07C8A
:10182700008D3A753F15755903755AF4E537C3941A
:101837000B50051211888006900487E0F537E537CD
:1018470075F0FFA4FFAEF09000E1E08E048F05FF76
:10185700127075ED900074F0E56675F078A4FFAE30
:10186700F074FF8E048F05FF1270758C598D5A74B2
:10187700028C068D071200398F37AC59AD5A7404A4
:10188700FF1270A08D3A753F04755906755A28E501
:1018970037C3941D500512118880069006CDE0F5D8
:1018A70037AE2AAF2BE5372FFF50010E7464127045
:1018B700C88E2A8F2B90008DE0B4025DE56175F02C
:1018C70064A4FFAEF074081200398E5B8F5C740558
:1018D7008E048F05FF1270758D37AE5BAF5C740594
:1018E7008E048F05FF1270A08D3A753F0575590557
:1018F700755ADEE537C39413500512118880069098
:101907000679E0F537AE2AAF2BE5372FFF50010EEA
:1019170074641270C88E2A8F2B9000CFE0707F906E
:101927000053E075F00A84FF7E008F37900053E084
:1019370075F00A84ADF07C008D3A753F0A7559053C
:10194700755AC0E537C3940E50051211888006906A
:101957000656E0F537E537900079F09000EEE0B4F1
:10196700023C900053E075F00A84FF7E008F3790A9
:101977000053E075F00A84ADF07C008D3A753F0A9C
:10198700755905755ACFE537C3940E50051211885E
:101997008006900665E0F537E53790007AF02290EB
:1019A7000096E0B401179008EBE0252BFFAE2A5014
:1019B700010E9000EAE01270C88E2A8F2B90010E5C
:1019C700E0B4011490010FE0A851B80004955250FB
:1019D70007E55FC39560400280139000B8E0252BB0
:1019E700FFAE2A50010E8E2A8F2B021E0D900096F5
:1019F700E0B40306A228B3B3400280509008F5E094
:101A070070109008EEE0C39405A851B800069552EF
:101A1700400280109000B8E0252BFFAE2A50010E3F
:101A27008E2A8F2B9008F5E0600D9008EEE0A85104
:101A3700B800069552400280109000B8E0252BFFB1
:101A4700AE2A50010E8E2A8F2B021E0D900090E0B9
:101A5700B402028003021E0D900093E0602FE56739
:101A6700D394464028900012E0FEA3E0FF9000CEFA
:101A7700E075F003A4FDACF0EFD39DEE9C400E9013
:101A870000F2E0A851B80005D395525003021E0D8D
:101A97009000C3E0B403028003021C5585615A75A8
:101AA700590090009AE0A851B800049552500E9042
:101AB700009BE0A859B80005D3955A5003021C5261
:101AC700E56175F002A4FFAEF074158E048F05FF73
:101AD7001270758C068D07900618120048FEE0FFFD
:101AE700EE900092E0FEEF8E0088F0A4FFAEF07457
:101AF700648E048F05FF1270758C598D5A900053B0
:101B0700E075F018A4FFAEF09000D9E08E048F05C1
:101B1700FF1270758C068D07900630120048AE597B
:101B2700AF5AE012708574648E048F05FF127075CA
:101B37008C598D5AE565A859B80005D3955A5003B5
:101B4700021BC9E565C3955AFFE49559FE8E598F67
:101B57005A7428BE00039F500C755A287559007493
:101B67000D900054F0AE59AF5A900093E012708573
:101B770074288E048F05FF1270758C598D5A900842
:101B870090E0FEA3E0FF740A8E048F05FF127075C4
:101B97008D068C07AC59AD5ACFCECF120003740A0D
:101BA7008E048F05FF1270758C598D5A900890E03E
:101BB700FEA3E0FF1270D0900890EEF0A3EFF002C2
:101BC7001C52E565A859B80004955A507EAE59AF26
:101BD7005AE5651270C88E598F5A7428BE00039F44
:101BE700500C755A28755900740D900054F0AE5971
:101BF700AF5A900093E012708574288E048F05FF0A
:101C07001270758C598D5A900890E0FEA3E0FF740E
:101C17000A8E048F05FF1270758D068C07AC59ADBF
:101C27005ACFCECF120003740A8E048F05FF1270AD
:101C3700758C598D5A900890E0FEA3E0FFEF2DFDBB
:101C4700EE3CFC900890ECF0A3EDF0021E0D900026
:101C5700DBE0855FF0A4FFAEF074051270857407B2
:101C67001200398E598F5A90009AE0A851B8000493
:101C77009552501290009BE075F002A4FDACF0EF76
:101C8700C39DEE9C4003021E0DE55F75F00B84FFBC
:101C97007E00900618120048FEE0FFEE900092E0EA
:101CA700FEEF8E0088F0A4FFAEF074648E048F05FB
:101CB700FF1270758C598D5A900053E075F018A477
:101CC700FFAEF09000D9E08E048F05FF1270758C7F
:101CD700068D07900630120048AE59AF5AE01270D1
:101CE7008574648E048F05FF1270758C598D5AE5C3
:101CF70065A859B80005D3955A5003021D84E565B8
:101D0700C3955AFFE49559FE8E598F5A7428BE0021
:101D1700039F500C755A28755900740D900054F0A4
:101D2700AE59AF5A900093E012708574288E048FD5
:101D370005FF1270758C598D5A900890E0FEA3E04C
:101D4700FF740A8E048F05FF1270758D068C07AC21
:101D570059AD5ACFCECF120003740A8E048F05FFF8
:101D67001270758C598D5A900890E0FEA3E0FF120F
:101D770070D0900890EEF0A3EFF0021E0DE565A875
:101D870059B80004955A507EAE59AF5AE56512709E
:101D9700C88E598F5A7428BE00039F500C755A2855
:101DA700755900740D900054F0AE59AF5A900093D6
:101DB700E012708574288E048F05FF1270758C5998
:101DC7008D5A900890E0FEA3E0FF740A8E048F05F9
:101DD700FF1270758D068C07AC59AD5ACFCECF1256
:101DE7000003740A8E048F05FF1270758C598D5A83
:101DF700900890E0FEA3E0FFEF2DFDEE3CFC90087D
:101E070090ECF0A3EDF0229000EEE0B4027BE55FEA
:101E170075F00884FF7E008F37E55F75F00884ADA5
:101E2700F07C008D3A753F08755901755AE0E53722
:101E3700C3943F50051211888006900287E0F5375A
:101E4700E537900892F8E4F0E8A3F0900892E0FEF6
:101E5700A3E0FFAC2AAD2B12000374648E048F0538
:101E6700FF127075900892ECF0A3EDF090008BE0F4
:101E77008C068D0712708574648E048F05FF1270AF
:101E870075900892ECF0A3EDF0900890E0FEA3E0C7
:101E9700FFAC2AAD2B12000374648E048F05FF126A
:101EA7007075900890ECF0A3EDF090008BE08C0635
:101EB7008D0712708574648E048F05FF12707590FC
:101EC7000890ECF0A3EDF0A204401DAE51AF5274A0
:101ED70005BE00039F5002D204E561D394CC4008AD
:101EE700D2027411900054F0229000EDE0B4020881
:101EF7009000DBE0640B60028045900890E0FEA351
:101F0700E0FFE56B12708574E78E048F05FF127092
:101F170075900890ECF0A3EDF09000EEE0B4021F8E
:101F2700900892E0FEA3E0FFE56B12708574E78EE0
:101F3700048F05FF127075900892ECF0A3EDF090F6
:101F470000ADE05402601B9000A4E0A851B8001255
:101F5700D39552400DA204B3B35007E561C3949AD9
:101F67004002805FAE34AF359000A2E075F002A466
:101F7700FDACF0EF2DFDEE3CFC74022DFD50010C85
:101F8700E561BC003ED39D403A754301A22F403323
:101F97009000A3E075F05EA4FDACF07405FF12702D
:101FA700758C5B8D5C124A74900890E0FEA3E0FF8D
:101FB7009000A3E02FFF50010E900890EEF0A3EFE2
:101FC700F0D22FE561A834B8000495355002C22F2E
:101FD700856135753400E54370030220E690010002
:101FE700E0C3954350030220D8900110E0C3940248
:101FF7004003022082E56775F00A84FF7E009005A2
:1020070088120048E0F55A755900AE59AF5A90004A
:10201700A3E012708574648E048F05FF1270758CAF
:102027005B8D5C900100E004C395438C068D07121D
:102037007085900100E08E048F05FF1270758C5B30
:102047008D5C900890E0FEA3E0FFEF2DFDEE3CFCD9
:10205700900890ECF0A3EDF09000EEE0B4021A9037
:102067000892E0FEA3E0FFAA5BAB5CEF2BFBEE3A26
:10207700FA900892EAF0A3EBF08056900100E00492
:10208700C39543854BF0A4FFAEF0900100E08E04AA
:102097008F05FF1270758C5B8D5C900890E0FEA336
:1020A700E0FFEF2DFDEE3CFC900890ECF0A3EDF087
:1020B7009000EEE0B4021A900892E0FEA3E0FFAAB7
:1020C7005BAB5CEF2BFBEE3AFA900892EAF0A3EBDE
:1020D700F00543900100E0C395435003754300901A
:1020E70000ADE05401601B9000A1E0A851B80012B8
:1020F700D39552400DA204B3B35007E55FC394CC08
:102107004002806090009FE075F003A4FFAEF0E509
:10211700402FFF50010E74032FFF50010EE55FBEE5
:102127000042D39F403E754401A22F40379000A044
:10213700E075F05EA4FFAEF074058E048F05FF1204
:1021470070758C5B8D5C124A74900890E0FEA3E07A
:10215700FF9000A0E02FFF50010E900890EEF0A333
:10216700EFF0D22FE55FC395405002C22F855F4045
:10217700E5447003022280900101E0C395445003B7
:10218700022272900110E0C39402400302221CE570
:102197006775F00A84FF7E00900588120048E0F515
:1021A7005A755900AE59AF5A9000A0E01270857465
:1021B700648E048F05FF1270758C5B8D5C90010136
:1021C700E004C395448C068D07127085900101E0E9
:1021D7008E048F05FF1270758C5B8D5C900890E004
:1021E700FEA3E0FFEF2DFDEE3CFC900890ECF0A382
:1021F700EDF09000EEE0B4021A900892E0FEA3E042
:10220700FFAA5BAB5CEF2BFBEE3AFA900892EAF081
:10221700A3EBF08056900101E004C39544854CF090
:10222700A4FFAEF0900101E08E048F05FF127075D8
:102237008C5B8D5C900890E0FEA3E0FFEF2DFDEE38
:102247003CFC900890ECF0A3EDF09000EEE0B402B7
:102257001A900892E0FEA3E0FFAA5BAB5CEF2BFBB2
:10226700EE3AFA900892EAF0A3EBF00544900101E8
:10227700E0C395445003754400900890E0FEA3E046
:10228700FF9000B2E0BE00039F500D9000B2E090B7
:102297000890F8E4F0E8A3F09000EEE0B4021290A2
:1022A7000892E0FEA3E0FF9000B2E0BE00059F4069
:1022B70002800D9000B2E0900892F8E4F0E8A3F0F5
:1022C700229000EEE0B401028003022416A204B3B8
:1022D70050030223FD9000B9E0B4017A900890E022
:1022E700FEA3E0FFAC51AD52120003743C8E048F85
:1022F70005FF1270759000C9E0BC00159D40129053
:102307000890E0FEA3E0FF9000CBE0BE00039F50E3
:1023170002D203900890E0FEA3E0FFAC51AD521249
:102327000003743C8E048F05FF1270759000C9E09E
:10233700C3940ABC001AD39D4016900890E0FEA3F0
:10234700E0FF9000CBE0C39405BE0004D39F50028A
:102357008002C203807A900890E0FEA3E0FFAC51B0
:10236700AD5212000374788E048F05FF12707590BA
:1023770000C9E0BC00159D4012900890E0FEA3E064
:10238700FF9000CBE0BE00039F5004D20380419032
:102397000890E0FEA3E0FFAC51AD52120003747841
:1023A7008E048F05FF1270759000C9E0C3940ABCB4
:1023B700001AD39D4016900890E0FEA3E0FF90001E
:1023C700CBE0C39405BE0004D39F50028002C20332
:1023D700A203B34021900890E0FEA3E0FF9000CA5B
:1023E700E012708574648E048F05FF127075900873
:1023F70090ECF0A3EDF0A203B3400CA233400674B7
:1024070024900054F0D233A2034002C2338002C2A8
:102417000390004FE06006A204B3B3400280199016
:102427000890E0FEA3E0FF90004FE02FFF50010E61
:10243700900890EEF0A3EFF0A201B34006A202B31A
:10244700B3500990001AE4F0A3F0802D900890E0B3
:10245700FEA3E0FF7400D39F74019E401190089083
:10246700E0F8A3E090001AC8F0A3C8F0800B74FF4F
:1024770090001AF8E4F0E8A3F09000D0E0C39404C9
:10248700400C9008F2E0C3940240030225709000CC
:10249700B9E0B40147900890E0FEA3E0FF745E1234
:1024A700708574058E048F05FF127075900890EC87
:1024B700F0A3EDF09000EEE0B4021F900892E0FE6A
:1024C700A3E0FF745E12708574058E048F05FF12FA
:1024D7007075900892ECF0A3EDF08045900890E0BD
:1024E700FEA3E0FF745E127085740A8E048F05FFE9
:1024F700127075900890ECF0A3EDF09000EEE0B448
:10250700021F900892E0FEA3E0FF745E12708574CC
:102517000A8E048F05FF127075900892ECF0A3EDF8
:10252700F0900890E0FEA3E0FF7402BE000CD39F7A
:102537004008752902752800800A900890E0F52860
:10254700A3E0F529900892E0FEA3E0FF7402BE0025
:102557000CD39F4008752D02752C00800A900892B5
:10256700E0F52CA3E0F52D8046900890E0FEA3E06F
:10257700FF7401BE000CD39F400875290175280020
:10258700800A900890E0F528A3E0F529900892E0EA
:10259700FEA3E0FF7401BE000CD39F4008752D0118
:1025A700752C00800A900892E0F52CA3E0F52D9099
:1025B7000018E528F0A3E529F0A236B34009C201C7
:1025C70090001AE4F0A3F022900053E090038812E1
:1025D70070B6E0F541754264900053E0FE9000C488
:1025E700E0D39E4037E55F75F00884FF7E008F37A4
:1025F700E55F75F00884ADF07C008D3A753F08758E
:102607005903755A96E537C3941F500512118880F0
:102617000690043DE0F5378537428035E55F75F074
:102627000884FF7E008F37E55F75F00884ADF07C86
:10263700008D3A753F08755903755AB6E537C39447
:102647001F5005121188800690045DE0F537853725
:1026570042229000FAE0F53C753F11755904755A0E
:1026670000AE51AF52E53C75F00FA4FDACF0EDD3D1
:102677009FEC9E4021E53C8E048F05FF127075ED9F
:1026870075F010A4FFAEF0E55F75F01184FD7C00D6
:10269700ED2FF53D800EE55F75F01184FF7E00EFAD
:1026A70024F0F53D853D37E55F75F01184AFF07E89
:1026B700008F3A12118885373EAE51AF529000FA1B
:1026C700E075F00FA4FDACF0EDD39FEC9E402875AC
:1026D7005904755A10853D37121188853E3885375C
:1026E70039AE51AF52E53C8E048F05FF1270A08DB5
:1026F7003A853C3B121202853741754264229000AD
:10270700FAE0F53C753F11755904755A00AE51AFA3
:1027170052E53C75F00FA4FDACF0EDD39FEC9E4065
:1027270021E53C8E048F05FF127075ED75F010A43E
:10273700FFAEF0E56175F01184FD7C00ED2FF53DEE
:10274700800EE56175F01184FF7E00EF24F0F53D02
:10275700853D37E56175F01184AFF07E008F3A1241
:10276700118885373EAE51AF529000FAE075F00FF1
:10277700A4FDACF0EDD39FEC9E4028755904755A23
:1027870010853D37121188853E38853739AE51AFF0
:1027970052E53C8E048F05FF1270A08D3A853C3BB5
:1027A7001212028537417542649000F5E0B404794E
:1027B700900053E0FE9000C4E0D39E4037E55F757C
:1027C700F00884FF7E008F37E55F75F00884ADF071
:1027D7007C008D3A753F08755903755A96E537C3DE
:1027E700941F5005121188800690043DE0F5378547
:1027F70037428035E55F75F00884FF7E008F37E547
:102807005F75F00884ADF07C008D3A753F08755907
:1028170003755AB6E537C3941F5005121188800611
:1028270090045DE0F5378537422290008EE0B401D1
:102837003BE56775F00A84FF7E008F37E56775F023
:102847000A84ADF07C008D3A753F0A755905755AB3
:1028570012E537C39411500512118880069005AB15
:10286700E0F537E5422537C39464F54290008FE0E1
:10287700B4013BE56875F00A84FF7E008F37E56891
:1028870075F00A84ADF07C008D3A753F0A755905DD
:10289700755A7EE537C3941150051211888006904A
:1028A7000617E0F537E5422537C39464F542E5415D
:1028B7002542F536900096E0B402109008EAE0252C
:1028C70036FE9000EAE0F4042EF5369000EDE0D3F2
:1028D70094014040E56BC394E7501D74E7C3956BC3
:1028E700FE9008ECE08E00F5F0E884FF7E008F375D
:1028F700E5362537F536801CE56BC394E7FE90086F
:10290700ECE08E00F5F0E884FF7E008F37E536C3F4
:102917009537F536A2044006E5412464F536E536D9
:10292700D394644009E536C39464F536800375365D
:10293700009000C6E0C3953650069000C6E0F53615
:1029470022D201900077E0A851B800049552503E7A
:10295700900077E0A851B800049552500375360FE0
:10296700900077E004A851B80004955250037536DB
:1029770007900077E02402A851B80004955250024E
:10298700C201900077E060067409900054F0C22EEF
:102997007E017F009000CCE01270859000DBE08E16
:1029A700048F05FF127075E55FBC000CD39D4008CE
:1029B700D236740A900054F090008EE0B40109906A
:1029C70000CDE0C39567400280159000DFE0A85175
:1029D700B8000495525002C201740B900054F09055
:1029E700008EE0B40107E567C394644002801D9040
:1029F7000125E0600D900125E0A851B80006955229
:102A070040028008C201740B900054F0A2014003F9
:102A1700753600C23590010EE0B4011490010FE045
:102A2700A851B8000495525007E55FC3956040026E
:102A3700802A9000B7E0D3941D400B9000B7E0C305
:102A4700941EF5368003753600A23240087415903F
:102A57000054F0D235D232D230022B42C230C232C9
:102A6700900096E0B40306A228B3B34003022B42BA
:102A77009008EEE0C39405A851B80004955250069B
:102A87009008F5E06002801F9000B7E0D3941D40E6
:102A97000B9000B7E0C3941EF536800375360074BB
:102AA7000C900054F0D2359008EEE0A851B800041D
:102AB700955250069008F5E07002801F9000B7E02D
:102AC700D3941D400B9000B7E0C3941EF5368003E6
:102AD700753600740C900054F0D2359008EEE0A8DB
:102AE70051B80004955250319000D5E0B40228D275
:102AF7002E9008F4E0FE9008F5E0D39E500690086B
:102B0700F5E0700280099008F4E4F0C22E80069088
:102B170008F4E004F08002C2019008EEE02405A862
:102B270051B80004955250139000D5E0B4020A90B2
:102B370008F5E07002D22E8002C201A22DB3402711
:102B47009000B7E0D3941D400B9000B7E0C3941EEC
:102B5700F5368003753600A2314006741090005494
:102B6700F0D231D2358002C23185366C9000B7E0A1
:102B7700D3941D4018900085E02536FE900053E061
:102B870075F01E84FC7F00EE2CF5368029A235B344
:102B97004008900085E0F536801C900087E02536D8
:102BA700FE900085E02EFE900053E075F01E84FC39
:102BB7007F00EE2CF536A236B34005D22E756C0099
:102BC70022900053E075F00584FF7E008F37900058
:102BD70053E075F00584ADF07C008D3A753F0575BF
:102BE7005903755AD69000D9E01475F00584FF7E15
:102BF70000E537BE00039F5005121188800BE537AB
:102C070090045E1270B6E0F537E5379008EDF09066
:102C170008EDE0FE9000C8E0C39E50089000C8E0B1
:102C27009008EDF09000B7E0D3941D401E9008ED9A
:102C3700E0FE900085E02EFE900053E075F01E84C4
:102C4700FC7F00EE2C9008EDF08031A235B3400AEE
:102C5700900085E09008EDF080229008EDE0FE906E
:102C67000087E02EFE900085E02EFE900053E07571
:102C7700F01E84FC7F00EE2C9008EDF02290008E71
:102C8700E0B40136E56775F00A84FF7E0090058899
:102C9700120048E0F546E546D394644010E546C384
:102CA700946475F00F84FF7E008F4680037546009D
:102CB7009000ABE02546F54680069000ABE0F54670
:102CC70022E56775F00A84FF7E00900588120048A8
:102CD700E0C394694007E567D3946440559000F5D5
:102CE700E0C39403502690088AE0FEA3E0FF740433
:102CF700120039E55F127085740F8E048F05FF127D
:102D07007075900888ECF0A3EDF0802490088AE0B5
:102D1700FEA3E0FF7404120039E561127085740F99
:102D27008E048F05FF127075900888ECF0A3EDF004
:102D3700800F90088AE0F8A3E0900888C8F0A3C83D
:102D4700F0A204401A90088AE0FEA3E0FF74031281
:102D570070857401120039900888EEF0A3EFF090A7
:102D6700009EE0B40262E56AC3944175F00584FFF2
:102D77007E008F37E56A75F00584ADF07C008D3AEB
:102D8700753F05755906755A14E537C394175005ED
:102D970012118880069006AFE0F537900888E0FEAC
:102DA700A3E0FF740A8E048F05FF127075E5378C58
:102DB700068D07127085740A8E048F05FF127075D1
:102DC700900888ECF0A3EDF0900888E0FEA3E0FF00
:102DD70090088EE0FCA3E0FDEDD39FEC9E400F90A2
:102DE700088EE0F8A3E0900888C8F0A3C8F022E5B1
:102DF7000875F004A4FFAEF09006CB120048E090EF
:102E07003C4BF8282873804C85527380479000DB31
:102E1700E0855FF0A4FFAEF074081200398F73806D
:102E270033856173802E8567738029856873802455
:102E3700856973801F856A73801A856B7380158512
:102E470066738010856573800B856C7380069000B0
:042E57001BE0F57314
:103C4B00022E0D022E0F022E14022E28022E2D02F2
:103C5B002E32022E37022E3C022E41022E46022E0F
:073C6B004B022E50022E5502
:102E5B00E50875F004A4FFAEF09006CC120048E52F
:102E6B000875F004A4FFAEF0E0FC9006CD1200480C
:102E7B00ECFEE0FFEEC39F4003022F63E50875F005
:102E8B0004A4FFAEF09006CB120048E0B40441E579
:102E9B000875F004A4FFAEF09006CD120048E0C315
:102EAB009573500AE508F50CD39237123DA6E50849
:102EBB0075F004A4FFAEF09006CC120048E0D39559
:102ECB0073400AE508F50CC39237123DA6022F6139
:102EDB00E50875F004A4FFAEF09006CC120048E0B4
:102EEB00C395735015E50875F004A4FFAEF090067A
:102EFB00CD120048E0D395735002800AE508F50C1B
:102F0B00D39237123DA6E50875F004A4FFAEF090FE
:102F1B0006CC120048E0D395735015E50875F00404
:102F2B00A4FFAEF09006CD120048E0C39573500A93
:102F3B00E508F50CC39237123DA69006D3E0B40119
:102F4B00099000E7E0D395615002800A7402F50CFA
:102F5B00C39237123DA6806AE50875F004A4FFAE54
:102F6B00F09006CC120048E0D395734015E5087538
:102F7B00F004A4FFAEF09006CD120048E0C39573A9
:102F8B004002800AE508F50CC39237123DA6E5080E
:102F9B0075F004A4FFAEF09006CC120048E0C39588
:102FAB00734015E50875F004A4FFAEF09006CD1242
:102FBB000048E0D39573400AE508F50CD39237121D
:102FCB003DA622AE2EAF2F74C9BE000CD39F400876
:102FDB00782E1270D80230E8752F01752E00AE5185
:102FEB00AF52E546BE000DD39F40099000BDE0D324
:102FFB00954740028023754700E546C39552F5730C
:10300B009000C0E0D395454008E5452573F5458014
:10301B00069000C0E0F54580020547900099E0D38B
:10302B009561401CE55FC395604015AE51AF52E50D
:10303B0046BE00039F50099000BEE0D39548400266
:10304B00806E9008EFE0A851B800049552500375BC
:10305B004A009008EFE0A851B8000BD395524006F8
:10306B00E5529008EFF0E54A7041E552C39546F5FD
:10307B0073E573D3940540037573059000BFE0C3EC
:10308B0095455007E573C3954540028009E545C357
:10309B009573F54580069000BFE0F5459000BFE0C5
:1030AB00D3954540069000BFE0F54575480080027A
:1030BB000548E54A7016900099E0C39561500DE5FF
:1030CB00462405A851B8000695524002800F900087
:1030DB00ACE0F545754A0174789008EFF022AE2EFE
:1030EB00AF2F74E9D39F74039E4008782E1270D8CB
:1030FB0002328F752F01752E00754532A229402A99
:10310B007545199000ACE075F002A4FFAEF0E547F1
:10311B00BE0006D39F4002D2290547754A03747837
:10312B009008EFF0754900023276AE51AF52E5468A
:10313B006F4E7003023276E546BE000DD39F4009F9
:10314B009000BDE0D395474002800F754700E54ADC
:10315B00C394035003754519800DE546C39552F58D
:10316B0073E5472573F547900099E0D39561400EC1
:10317B009008EFE0A851B80007D395524002800C9D
:10318B0005499000ACE0B54903754A00E54AB40324
:10319B0006A204B3B34002800A0549E549B43C03D7
:1031AB00754A02E54AB402299008EFE0A851B8002D
:1031BB000ED395524009E5529008EFF075490090F7
:1031CB000099E0C39561500975490074789008EF38
:1031DB00F0E54A705A900099E0D39561401CE55F89
:1031EB00C395604015AE51AF52E546BE00039F50EC
:1031FB00099000BEE0D395484002800875480075E1
:10320B00454B8028E552C39546F573E573D394057A
:10321B004003757305900099E0D395614008E5482C
:10322B002573F5488006E5482406F548754900E501
:10323B004A7016900099E0C39561500DE546240540
:10324B00A851B80006955240028003754A01E54A21
:10325B00B4011875451905499000ACE0B5490675E0
:10326B004A0275490074789008EFF0A202B340034C
:10327B00754532E54575F00AA4FFAEF0900894EE63
:10328B00F0A3EFF022E56F903C72F8282873023C14
:10329B000B900091E070030235BA9000C7E0B401C7
:1032AB00028003023450900051E0655E6009E552E4
:1032BB004551600302344D7E017F00E5BE127085DF
:1032CB00E5BD2FFF50010E8E598F5A9000C5E0B40B
:1032DB00461B740E127085900076E08E048F05FFEE
:1032EB00127075900898ECF0A3EDF0801DAE59AFFD
:1032FB005A7410127085900076E08E048F05FF12C1
:10330B007075900898ECF0A3EDF0E56B600FE56B32
:10331B00C394FE50089000EDE0640260028064905C
:10332B0000DBE0B40B1F900898E0FEA3E0FF74E70E
:10333B00127085E56B8E048F05FF127075900898DF
:10334B00ECF0A3EDF09000DBE0D3940B4008900081
:10335B00C3E064046002802B900898E0FEA3E0FFBA
:10336B0090089CE0FCA3E0FDEFD39DEE9C400D127A
:10337B0070D0900898EEF0A3EFF08007900898E4D7
:10338B00F0A3F0900898E0FEA3E0FFEFD39400EEDB
:10339B0094014008D2367426900054F0A236B3B391
:1033AB00502C7E057F009000DBE08E048F05FF1212
:1033BB007075900898E0FEA3E0FFEFC39DEE9C4074
:1033CB000FAC51AD52740FBC0004D39D5002800260
:1033DB00C236900091E0B4022790089AE0FEA3E079
:1033EB00FF900898E0FCA3E0FDEF2DFDEE3CFC7494
:1033FB00018C068D07120039900898EEF0A3EFF0C0
:10340B00900898E0FEA3E0FF90089AE0FCA3E0FD93
:10341B00EDD39FEC9E4004D22C8002B22C900898E6
:10342B00E0F8A3E090089AC8F0A3C8F09000C3E0BE
:10343B0064016006A22CB3B340028006900899E0A9
:10344B00F55F0235B8D22C7E017F00E5BE12708588
:10345B00E5BD2FFF50010E8E598F5A9000C5E0B479
:10346B00461B740E127085900076E08E048F05FF5C
:10347B00127075900898ECF0A3EDF0801DAE59AF6B
:10348B005A7410127085900076E08E048F05FF122F
:10349B007075900898ECF0A3EDF0E56B600FE56BA1
:1034AB00C394FE50089000EDE064026002806490CB
:1034BB0000DBE0B40B1F900898E0FEA3E0FF74E77D
:1034CB00127085E56B8E048F05FF1270759008984E
:1034DB00ECF0A3EDF09000DBE0D3940B40089000F0
:1034EB00C3E064046002802B900898E0FEA3E0FF29
:1034FB0090089CE0FCA3E0FDEFD39DEE9C400D12E9
:10350B0070D0900898EEF0A3EFF08007900898E445
:10351B00F0A3F0900898E0FEA3E0FFEFD39400EE49
:10352B0094014008D2367426900054F0A236B3B3FF
:10353B00502C7E057F009000DBE08E048F05FF1280
:10354B007075900898E0FEA3E0FFEFC39DEE9C40E2
:10355B000FAC51AD52740FBC0004D39D50028002CE
:10356B00C236900091E0B4022790089AE0FEA3E0E7
:10357B00FF900898E0FCA3E0FDEF2DFDEE3CFC7402
:10358B00018C068D07120039900898EEF0A3EFF02E
:10359B00900898E0F8A3E090089AC8F0A3C8F090C0
:1035AB0000C3E064016006900899E0F55F80037545
:1035BB005F0090008DE07006756F0302329075BB53
:1035CB0018023C0B023C0B90008DE070030237435A
:1035DB007E017F00E5BE127085E5BD2FFF50010E09
:1035EB008E598F5A9000D3E0B4010F7E0F7FFFAC42
:1035FB0059AD5A1270D08E598F5A9000F8E0B40220
:10360B0045AE59AF5A900024E0FCA3E0FDEDD39FEB
:10361B00EC9E400A900024E559F0A3E55AF0AE5910
:10362B00AF5A900026E0FCA3E0FDEFD39DEE9C404B
:10363B000A900026E559F0A3E55AF0AE59AF5A743B
:10364B00041200398F619000F8E0704CAE59AF5AFC
:10365B00900024E0FCA3E0FDEFD39DEE9C4009120B
:10366B0070D08E598F5A8006755A00755900AE5915
:10367B00AF5A74101270859000F7E08E048F05FF1F
:10368B001270758C598D5A74FFBC0009D39D40057F
:10369B00855A6180037561FE9000C3E0B40102801E
:1036AB0003023741A204B3B3500E900097E0A85128
:1036BB00B80005D39552500280719000D4E085611B
:1036CB00F0A4FFAEF074648E048F05FF1270758C3E
:1036DB00598D5AE56B6016E56BC394FE500F900045
:1036EB00EDE0B402089000DBE0640B60028017AEE3
:1036FB0059AF5A74E7127085E56B8E048F05FF1274
:10370B0070758C598D5AAE59AF5A900898E0FCA33E
:10371B00E0FDEDD39FEC9E4005855A5F800BA22CFC
:10372B00B34006900899E0F55F800BA22CB34006DE
:10373B00900899E0F55F8003756100900090E07050
:10374B0006756F0502329075BB19023C0B023C0BE0
:10375B00900090E070030237FBE55ED3955D40036C
:10376B000237F9900022E0FEA3E0FFE5651270C876
:10377B00900022EEF0A3EFF07E017F00E5BE127009
:10378B0085E5BD2FFF50010E8E598F5A9000FDE03D
:10379B007013740A12708574518E048F05FF1270AA
:1037AB00758D658019AE59AF5A740A1270858F04E6
:1037BB008E057E017F95CDCCCD126F738F65E56540
:1037CB00D394644003756564900022E0FEA3E0FF90
:1037DB00E5652FFF50010E900022EEF0A3EFF09065
:1037EB000094E0048E048F05FF1270758D658003C5
:1037FB007565329000E0E07006756F0702329075C8
:10380B00BB13023C0B023C0B9000E0E0604A7E01D4
:10381B007F00E5BE127085E5BD2FFF50010E8E595E
:10382B008F5A74041200398F669000E2E08566F0BF
:10383B00A4FDACF07464FF1270758D669000E1E02E
:10384B008566F0A4FFAEF074FF8E048F05FF127037
:10385B0075ED900075F0800375660090008EE0703A
:10386B0006756F0902329075BB17023C0B023C0BBD
:10387B0090008EE0B40102800302390F7E017F00BD
:10388B00E5BE127085E5BD2FFF50010E8E598F5A84
:10389B009008F0E060199008F0E014906A9812001C
:1038AB008CE493FC740193FDEDC39FEC9E4002806E
:1038BB00069008F0E014F09008F0E0C394B3501DAC
:1038CB00AE59AF5A9008F0E004906A9812008CE45D
:1038DB0093FC740193FDEFC39DEE9C400280069018
:1038EB0008F0E004F09008F0E0FE9000B4E08E00E9
:1038FB0088F0A4FFAEF074648E048F05FF12707510
:10390B008D67800375670090008FE07006756F0BF5
:10391B0002329075BB16023C0B023C0B90008FE001
:10392B00B4010280030239BB7E017F00E5BE127039
:10393B0085E5BD2FFF50010E8E598F5A9008F1E08F
:10394B0060199008F1E014906C0212008CE493FC67
:10395B00740193FDEDC39FEC9E400280069008F12D
:10396B00E014F09008F1E0C394B3501DAE59AF5A78
:10397B009008F1E004906C0212008CE493FC74014B
:10398B0093FDEFC39DEE9C400280069008F1E0048E
:10399B00F09008F1E0FE9000BAE08E0088F0A4FFF2
:1039AB00AEF074648E048F05FF1270758D68800302
:1039BB0075680075BB1F023C0B023C0B7E017F0040
:1039CB00E5BE127085E5BD2FFF50010E8E598F5A43
:1039DB00740912708574E68E048F05FF1270758D55
:1039EB006A900096E07006756F0F02329075BB15EA
:1039FB00023C0B023C0B900096E07003023B527EA4
:103A0B00017F00E5BE127085E5BD2FFF50010E8EC4
:103A1B00598F5A74041200398F69900096E0B401E3
:103A2B00159000EAE08569F0A4FFAEF07407120070
:103A3B0039EF9008EBF0900096E0B402159000EA95
:103A4B00E08569F0A4FFAEF07407120039EF90081F
:103A5B00EAF0900096E0B403028003023B3590003D
:103A6B00D7E07052E569C39419500FD2289000B675
:103A7B00E09008EEF09008F3E4F0E569D39464402D
:103A8B0004A2284002802D9008F3E004F09008F384
:103A9B00E0FE900129E0B5060B9008EEE004F090F3
:103AAB0008F3E4F09008EEE064966006900129E0DC
:103ABB007002C22880639000B6E070349000EAE098
:103ACB008569F0A4FFAEF074FF8E048F05FF1270B2
:103ADB0075ED9008EEF0AE51AF52741EBE0006D3DA
:103AEB009F4002D228E561D394E54002C228802989
:103AFB00E569C3940A500DAE51AF52741EBE00045B
:103B0B00D39F50028002D228E561D394E54002C2D4
:103B1B00289000B6E09008EEF09008EEE0C3940514
:103B2B00500674059008EEF0C22D900096E0B40498
:103B3B0014E569C394195002D22DE569D394324030
:103B4B0002C22DC22880037569009000EDE070065B
:103B5B00756F1102329075BB14023C0B023C0B903B
:103B6B0000EDE07003023BF87E017F00E5BE1270B2
:103B7B0085E5BD2FFF50010E8E598F5A900112E033
:103B8B007025EFD39421EE940E4005756BFF8015D5
:103B9B00AE59AF5A741012708574E38E048F05FF03
:103BAB001270758D6B8027AE59AF5AEFD39449EED7
:103BBB0094064005756BFF8015AE59AF5A74101201
:103BCB00708574638E048F05FF1270758D6BE56BBA
:103BDB0075F00BA4FFAEF09000DBE08E048F05FFB9
:103BEB0012707590089CECF0A3EDF08003756B00E0
:103BFB00900091E0600575BB1A800375BB188000BF
:103C720002329902329C0235CF0235D20237580203
:103C8200375B02381002381302387802387B023967
:103C9200240239270239C40239C70239FE023A0125
:093CA200023B67023B6A023C0B85
:103C0B00E56F75F00284AFF07E00EF4E7002D2ECE0
:033C1B00056F2210
:0970B6002582F5825002058322B7
:0F008C0025E050020583258250020583F582226C
:10705400EF2F500205832582F582E5833E2EF583CA
:017064002209
:1070C800CFC39FFF50011E22C3EF9DFFEE9CFE22FF
:0870D8000806B60002180622AA
:0D709300A3E004F070061270ACE004F022DF
:0E003900048007C3CE13CECF13CFD5E0F6223E
:106F7300BC000FBE0008ED8FF084FFADF022E4FEED
:106F8300FF22BE000DEF60FE54F0606F20E70302A6
:106F93007029EAC0E0EBC0E078017A0075F001EEF9
:106FA30020E710EF25E0FFEE33FE0AC5F023C5F01E
:106FB30030E7F0EA5407F9096A7A007B00600108B8
:106FC300C3EC9E40167004ED9F4010ED9FFDEC9EB8
:106FD300FCE5F0CA4ACA03F5F08005E5F003F5F0D5
:106FE300C3EE13FEEF13FFD9D77908CACBCAD8D0A3
:106FF300EAFEEBFFD0E0FBD0E0FA22EC8FF084FC5A
:10700300ED54F045F0C48FF084FEEDC454F045F028
:10701300C48FF084FDEEC4FE54F02DFFEE540F3CFC
:10702300FEADF07C0022790078008FF0EC7E082022
:10703300E70DC3CD33CD33C933C9C833C8DEF084BC
:1070430049F9E5F08FF0BE00E6FD7C00E9FFE8FEBC
:01705300221A
:0E708500F88FF0A4FFE5F0CE88F0A42EFE22D6
:10000300EF8DF0A4F9A8F0EF8CF0A428F8EE8DF0B2
:06001300A428FEE9FF2213
:10706500600D782B02706F007830D8FED5E0F822DD
:10707500EEC0E07E00126F73EFFDEEFCD0E0FE2265
:0C70A000EEC0E07E00126F73D0E0FE2214
:03001B0002001EC2
:0300530002005652
:03009B00020071EF
:030000000270BFCC
:0970BF0075817575D000024C13B7
:0B004800E5822FF582E5833EF5832260
:0A70AC000582D582021583158222A9
:10001E00C0E0C0F0C083C082C0D075D000124B3A91
:0B002E00D0D0D082D083D0F0D0E032E0
:10005600C0E0C0F0C083C082C0D075D000124B3D56
:10006600D0D0D082D083D0F0D0E032C0E0C0F0C093
:1000760083C082C0D075D000124B77D0D0D082D04A
:0600860083D0F0D0E0324F
:00000001FF
